:020000020000FC
:100000000C9481110C94490D0C945E0D0C946911A3
:100010000C94450D0C94460D0C94470D0C94480D12
:100020000C94320D0C94330D0C94340D0C94350D4E
:100030000C94360D0C94370D0C94380D0C94390D2E
:100040000C943A0D0C943B0D0C94730D0C943F0DD5
:100050000C9426100C946B100C94400D0C943D0DD8
:100060000C948E100C943C0D0C943E0D0C94440D8D
:100070000C94410D0C94420D0C94430D8954400B8B
:10008000B83630303000895A1C05783238303000AC
:10009000895A1C04B03234303000895A1C041A3298
:1000A00031303000895A1C03843138303000895790
:1000B0002E01F4313030300089572E00C820343002
:1000C000300089572E007D20323530001F28641102
:1000D0000001B0001D00B8000D001F2864110001D0
:1000E000B8000D00E0000D001F2864110001E000C1
:1000F0000D00E8001D001F2864110001BB001D0059
:10010000C3000D001F2864110001C3000D00D500BD
:100110000D001F2864110001D5000D00DD001D0039
:100120001F2864110001BC001D00C4000D001F2821
:1001300064110001C4000D00D4000D001F286411DB
:100140000001D4000D00DC001D001F286411000117
:10015000BD001D00C5000D001F2864110001C50071
:100160000D00D3000D001F2864110001D3000D0005
:10017000DB001D001F2864110001BE001D00C60029
:100180000D001F2864110001C6000D00D2000D00F3
:100190001F2864110001D2000D00DA001D001F2885
:1001A00064110001C0001D00C8000D001F2864116B
:1001B0000001C8000D00D0000D001F2864110001CF
:1001C000D0000D00D8001D001F2864110001C200DE
:1001D0001D00CA000D001F2864110001CA000D0097
:1001E000CE000D001F2864110001CE000D00D600C6
:1001F0001D001F2864110001C4001D00CB000D006C
:100200001F2864110001CB000D00CD000D001F2838
:1002100064110001CD000D00D5001D0006F1582726
:10022000102032304B0006F1580B54353830300076
:1002300006F1580578323830300006F1580514328E
:100240003630300006F158041A323130300006F1F1
:100250005803E8323030300006F15803843138302A
:10026000300006F15801F4313030300006F158000A
:10027000FA203530300006F15800C8203430300004
:1002800006F1580096203330300006F158007D20EA
:100290003235300006F158003E20313235001F283B
:1002A00064110001B0001D00B70010001F28641188
:1002B0000001B7001000E10010001F2864110001C8
:1002C000E1001000E8001D001F2864110001B200C9
:1002D0001D00B90010001F2864110001B9001000B2
:1002E000DF0010001F2864110001DF001000E6008D
:1002F0001D001F2864110001BC001D00C300100078
:100300001F2864110001C3001000D50010001F2831
:1003100064110001D5001000DC001D001F286411CD
:100320000001BD001D00C40010001F286411000161
:10033000C4001000D40010001F2864110001D40074
:100340001000DB001D001F2864110001BE001D000D
:10035000C50010001F2864110001C5001000D30063
:1003600010001F2864110001D3001000DA001D00E6
:100370001F2864110001BF001D00C60010001F28C7
:1003800064110001C6001000D20010001F28641183
:100390000001D2001000D9001D001F2864110001C7
:1003A000C0001D00C70010001F2864110001C70015
:1003B0001000D10010001F2864110001D1001000AE
:1003C000D8001D001F2864110001C1001D00C800D5
:1003D00010001F2864110001C8001000D000100098
:1003E0001F2864110001D0001000D7001D001F2835
:1003F00064110001C2001D00C90010001F28641113
:100400000001C9001000CF0010001F286411000176
:10041000CF001000D6001D001F2864110001C3008A
:100420001D00CA0010001F2864110001CA0010003E
:10043000CE0010001F2864110001CE001000D5006E
:100440001D001F2864110001C4001D00CB00100016
:100450001F2864110001CB001000CD0010001F28E0
:1004600064110001CD001000D4001D001F2864118C
:100470000001C5001D00CC0010001F286411000100
:10048000CC001000CC0010001F2864110001CC002B
:100490001000D3001D001F2864110001C6001D00BC
:1004A000CD0010001F2864110001CD001000CB000A
:1004B00010001F2864110001CB001000D2001D00A5
:1004C0001F2864110001CC002000CC000A001F2866
:1004D0006411020098000A00FF001D001F24BE00E6
:1004E00000001F2867010120504120566F6C747373
:1004F0002D3E20524620436F6D702D3E202020203F
:1005000020414C432D3E20202020205357522D3E89
:1005100020467764205077722D3E5265666C2050DD
:1005200077722D3E20504120437572722D3E4476E5
:100530007220437572722D3E0C1F286701011F2423
:10054000780002001F286701026B487A1F2861406B
:1005500000FF1F28614001FF0B1F286701040000F6
:100560000000001F286701020A2E000000FF0B1F79
:10057000286701042020202020000B1F2867010489
:100580000000001F286701021F243800020000003D
:10059000002E000000FF1F24000005001F28670137
:1005A0000154783A00000000002E00001F2864115A
:1005B000020098000800FF002E001F2442000500E2
:1005C0001F28670101523AFF4357285553422920FB
:1005D0004357284C534229205553422020202020A5
:1005E0004C53422020202020414D2020202020203C
:1005F000464D202020202020444947285553422999
:10060000444947284C5342291F24000005001F2855
:10061000670101583AFF1F24DA0007001F2867010D
:1006200001502DFF1F24CC0007001F286701015433
:1006300020FF1F24820005001F28670101FF1F24DF
:100640009A0004001F286701012A393A202020203F
:10065000202020343AFF1F248E0000001F2867014D
:10066000014C6F636BFF1F24000002001F2867010D
:10067000024F7574206F662062616E6421FF1F2433
:10068000000002001F2867010252414D207465736B
:1006900074207061737365646661696C65640C1FB6
:1006A00024000002001F2867010250726F6320734C
:1006B000796E63206661696C65641F24880001009F
:1006C0001F28670101202061416242634364446541
:1006D0004566466747684869496A4A6B4B6C4C6D8A
:1006E0004D6E4E6F4F7050715172527353745475FA
:1006F0005576567757785879597A5A30313233349B
:1007000035363738393F2C2E2F2D3D2B28262325E3
:100710002A3A3B21402924275F3C1F240000040083
:100720001F286701012020202020202020202020B9
:1007300020FF0C1F24200002001F286701044143F2
:10074000A7354147D3354148EC35414C0536414E3C
:100750001F36415072364152493641548C3642520E
:10076000AC36434100374342EE364346D136434C24
:10077000353743524637435357374354C0364355B2
:1007800024374358733744468B37444E8437445498
:100790009C374456B6374553CA374641ED37464233
:1007A000F93746440538464E21384652A13846535B
:1007B000DE384654BD384657FB3846588B394659C3
:1007C000B3394754D7394853003A4944163A494651
:1007D0001E3A49524A3849539B3A49585C3849595C
:1007E0006C384B4D043B4B53253B4B59453B4C43DD
:1007F000703B4C4B893B4C54A43B4D42BD3B4D435D
:10080000D63B4D44FD3B4D47323C4D524B3C4D5742
:100810009D3C4E42D73C4E54F33C4E570C3D50410C
:100820002E3D5043593D50449C3D504CBC3D504D95
:10083000D93D5052F83D50531C3E5054353E505710
:100840006F3E52418D3E5243B93E5244BE3E5246E7
:10085000E43E5247F73E524B143F524D3C3F5250FC
:10086000753F52547B3F5255CB3E52589F3F5342A7
:10087000B03F5343E73F534485405345B640534947
:10088000FE3F534DCD40535015405351E940535313
:1008900036405354574053566E40544306415446D5
:1008A0002541544C3641544D4F4154525E415458A9
:1008B000CF3F5550E6375641734156448C41564719
:1008C000BD415658CF4158431F42584424425854C2
:1008D000FB415855314258564A421F2458000000E7
:1008E000080843572855534229204357284C534260
:1008F000292055534220202020204C5342202020E4
:100900002020414D202020202020464D2020202046
:1009100020204449472855534229444947284C53ED
:1009200042291F240000070000044147432D04040E
:100930004175746F46617374536C6F774F666620B0
:100940001F243C00070000034E422D02046F666620
:10095000206F6E2020FF1F246C00070004045054F9
:10096000542050545443564F5820564F58431F2438
:100970008A000700000352782D02015452FF1F2401
:10098000AC000700000354782D02014142FF1F24F0
:100990009800010000074D657465723A20080A50FE
:1009A0004120566F6C74732020524620436F6D7047
:1009B000202020414C43202020202020205357522B
:1009C000202020202020204677642050777220208D
:1009D000205265666C20507772202050412043756C
:1009E000727220202044767220437572722020FF9C
:1009F0001F2498000200000D4D65746572206C691B
:100A00006768743A2008044F6666204C6F77314C53
:100A10006F77324C6F77334D6564314D6564324D7D
:100A200065643348696768FF1F2498000300000766
:100A300050205320423A20020A4F66662020202090
:100A40002020204F6E2020202020202020FF1F2447
:100A500098000400000F44697370207265732028A9
:100A6000487A293A20020231302031FF1F249800B1
:100A7000050000074E422050573A20030A53686F82
:100A8000727420202020204D656469756D2020201F
:100A9000204C6F6E67202020202020FF1F2498000C
:100AA0000100000E5054542D524620286D73293AEF
:100AB0002020FFF81F2498000200000A5043204124
:100AC0007564696F3A20020744697361626C654519
:100AD0006E61626C65201F2498000300000A547840
:100AE00020417564696F3A2002074D696320202018
:100AF000204C696E652020201F2498000400000C03
:100B00004C6F636B2074696D65723A2004054F6603
:100B1000662020313073202033307320203630732C
:100B200020201F2498000500000C506F776572206C
:100B3000736176653A2004054F6666202031356D75
:100B4000696E33306D696E36306D696E1F249800A2
:100B50000100000C50697463682028487A293A2003
:100B600001F81F2498000200000D53706565642091
:100B70002877706D293A2001F8FF1F2498000300A0
:100B8000000E456E68616E636564205353423A20DF
:100B900002034F6666204F6E1F2498000400000E6B
:100BA000464D2044657620286B487A293A20030375
:100BB000322E30342E30352E30FF1F2498000500A1
:100BC000000F4C6963656E736520636C6173733AE3
:100BD00020050245204120472054204E20FF1F249D
:100BE000980001000009565041202856293A20015A
:100BF000FAFF1F24980002000009495041202841B3
:100C0000293A2001FAFF1F249800030000094944F3
:100C100076202841293A2001FAFF1F249800040079
:100C20000009436D70286442293A2001FAFF1F240D
:100C3000980005000009414C43202856293A20011C
:100C4000FAFF1F249800010000095357522020206A
:100C5000203A2001FAFF1F2498000200000946777D
:100C600064202857293A2001FAFF1F249800030026
:100C70000009526566202857293A2001FAFF1F24EF
:100C800098000400000A202020202020202020207E
:100C9000020720202020202020202020202020208B
:100CA0001F2498000500000A20202020202020205A
:100CB000202002072020202020202020202020206B
:100CC00020201F2498000100000E564F5820676115
:100CD000696E3A2020202020FFF81F24980002008F
:100CE000000E564F582073656E733A202020202046
:100CF000FFF81F2498000300000E416E7469564FE0
:100D000058206761696E3A20FFF81F24980004009C
:100D1000000E564F5820646C792831306D73293A93
:100D2000FFF81F2498000500000A4D6963204269FE
:100D300061733A2002074F66662020202039205632
:100D40006F6C74731F24980001000005416D703AA8
:100D500020040C4E6F6E652020202020202020498A
:100D60006E74203130572020202020496E742031AD
:100D700030305720202020496E7420313030572BDE
:100D8000457874FF1F2498000200000C4B657965BC
:100D900072204D6F64653A20030549616D624149D7
:100DA000616D6242556C74696DFF1F2498000300E9
:100DB000000E4661726E73776F7274683A2020205D
:100DC00011034F6666202035202036202037202052
:100DD0003820203920313020313120313220313358
:100DE0002031342031352031362031372031382040
:100DF0003139203230FF1F2498000400000E534286
:100E00004920646C792831306D73293AFFF81F242A
:100E100098000500000E46424920646C79286D73E5
:100E2000293A2020FFF81F2498000100000E587670
:100E3000657274657220467265713A2017036F6699
:100E40006635302035322035342031343431343673
:100E50003232323232343432303432323432343468
:100E6000323634323834333034333234333434334A
:100E70003634333834343034343234343434343631
:100E8000343438FF1F249800020000094454523DB6
:100E90005054543A2002084E6F2020202020205920
:100EA00065732020202020FF1F2498000300000BE2
:100EB0004261756420726174653A2005062020390C
:100EC0003630302031393230302033383430302031
:100ED0003537363030313135323030FF1F2498000D
:100EE0000400000A48616E647368616B653A02072A
:100EF0002020204E6F6E654354532F5254531F24AD
:100F000098000500000D5475726E6F6E2064697351
:100F1000703A200204204F66664D736731FF1F242C
:100F200098000100000B5363616E20747269703A7F
:100F30002005062020202053352020202053362055
:100F400020202053372020202053382020202053D9
:100F500039FF1F2498000200000C5363616E207358
:100F6000746172743A20FFF81F2498000300000B8C
:100F70005363616E2073746F703A20FFF8FF1F2473
:100F800098000400000E4672657120696E6328485F
:100F90007A293A20090363686E20313031303020DD
:100FA000314B31304B31354B32304B32354B3530A4
:100FB0004BFF1F2498000500000D4477656C6C20E2
:100FC000286D73293A202005042031303020323535
:100FD00030203530303130303035303030FF1F2464
:100FE000980001000006526F6F663A20020B3730FE
:100FF0002E3030304D487A202037302E3435354D64
:10100000487A20201F24980002000008394D487AB1
:101010002D313A200109363030302020202020FFA9
:101020001F24980003000008394D487A2D323A20D9
:10103000090936303030202020202032383030204E
:101040002020202032343030202020202032313027
:101050003020202020203138303020202020203126
:10106000303030202020202034303020202020201C
:10107000203235302020202020206E6F6E65202009
:10108000202020FF1F24980004000008394D487AD2
:101090002D333A20090936303030202020202032EC
:1010A00038303020202020203234303020202020C2
:1010B00020323130302020202020313830302020A4
:1010C00020202031303030202020202034303020AB
:1010D00020202020203235302020202020206E6F3C
:1010E0006E652020202020FF1F24980005000008A6
:1010F000394D487A2D343A200909363030302020D5
:10110000202020323830302020202020323430304F
:101110002020202020323130302020202020313863
:10112000303020202020203130303020202020205E
:101130003430302020202020203235302020202044
:1011400020206E6F6E652020202020FF1F24980035
:101150000100000A3435354B487A2D313A20020718
:1011600032304B20202020353830302020201F24E2
:1011700098000200000A3435354B487A2D323A2067
:101180000E0732304B2020202035383030202020F0
:10119000323830302020203236303020202032319A
:1011A0003030202020323030302020203138303094
:1011B00020202031303030202020353030202020B9
:1011C00020343030202020203330302020202032A6
:1011D000353020202020313235202020206E6F6EC7
:1011E000652020201F2498000300000A3435354B69
:1011F000487A2D333A200E0732304B2020202035FC
:101200003830302020203238303020202032363024
:101210003020202032313030202020323030302039
:101220002020313830302020203130303020202034
:101230003530302020202034303020202020333022
:10124000302020202032353020202020313235201F
:101250002020206E6F6E652020201F24980004003F
:10126000000A3435354B487A2D343A200E07323097
:101270004B202020203538303020202032383030AC
:1012800020202032363030202020323130302020D3
:1012900020323030302020203138303020202031B2
:1012A00030303020202035303020202020343030A5
:1012B00020202020333030202020203235302020C4
:1012C0002020313235202020206E6F6E65202020B6
:1012D0001F2498000500000D46756C6C2044757045
:1012E0006C65783A2002044F6666204F6E2020FF1E
:1012F0001F249800010000095246472063616C3AA0
:1013000020FFF8FF1F2498000200000C41474320F3
:1013100043572F5353423A20FFF81F2498000300ED
:10132000000941474320414D3A2020FFF8FF1F2488
:10133000980004000008547820414C433A200209E8
:101340004F66662020202020204F6E202020202065
:1013500020201F2498000500000D54784257206378
:10136000616C205353423AFFF8FF1F24980001009C
:10137000000C464D2F494620746573743A200205CF
:101380004F666620204F6E2020201F249800020008
:10139000000B532F5077722063616C3A2002064F86
:1013A00066662020204F6E20202020FF1F249800FA
:1013B0000300000D54782053686628555342293A9B
:1013C00020FFF8FF1F2498000400000D54782053DC
:1013D0006866284C5342293A20FFF8FF1F249800E2
:1013E0000500000D5443584F20547765616B3A2037
:1013F00020FFF8FF1F249800010000054D7367319E
:101400003A010CFF1F249800020000054D7367325B
:101410003A010CFF1F249800030000054D73673349
:101420003A010CFF1F249800040000054D73673437
:101430003A010CFF1F249800050000054D73673525
:101440003A010CFF1F249800010000054D73673618
:101450003A010CFF1F249800020000054D73673706
:101460003A010CFF1F249800030000054D736738F4
:101470003A010CFF1F249800040000054D736739E2
:101480003A010CFF1F249800050000054D73313010
:101490003A010CFF1F2498000100000E436C7220DB
:1014A00074756E6572206D656D3A0203204E6F593A
:1014B00065731F2498000200000843202870462905
:1014C0003A2001F81F2498000300000E432073699E
:1014D00064653A202020202020200203416E7454AD
:1014E00078201F249800040000084C20286E48290A
:1014F0003A2001F81F2498000500000E466F726321
:101500006520726574756E653A2002034E6F20592E
:1015100065731F249800010000105072633120523F
:10152000657620412E30312E3234010120FF1F24F8
:10153000980002000009507263322052657620FF45
:10154000F8FF1F2498000300000A202020202020FC
:1015500020202020020720202020202020202020C2
:10156000202020201F2498000400000A2020202092
:1015700020202020202002072020202020202020A2
:101580002020202020201F2498000500000E5265F6
:101590002D70726F6772616D2075503A0203204E94
:1015A0006F5965731F248A00070000044644707851
:1015B0000000240033003E004A0052005A008B0015
:1015C000A700BA00C9000000240033003E004A0012
:1015D0005200E100ED00FE000F0124010000240094
:1015E00033003E004A0052003901440150015F01BE
:1015F00070010000240033003E004A0052008201C6
:101600008C019601A001AA010000240033003E00D5
:101610004A005200B401BE01C801D201E30100003A
:10162000240033003E004A005200F40100020C0284
:10163000180224020000240033003E004A00520039
:101640003502550268028E029A020000240033001F
:101650003E004A005200A602D502E702010312032F
:101660000000240033003E004A00520022033C03E5
:10167000470352036C030000240033003E004A007D
:10168000520082039503A303D5030704000024003E
:1016900033003E004A00520039044A048504C00465
:1016A000FB040000240033003E004A0052000B05FA
:1016B000150520052A053C050000240033003E00E6
:1016C0004A00520048055805690575058105000066
:1016D000240033003E004A0052008D0595059D050B
:1016E000A505AD050000240033003E004A0052006D
:1016F000B505BD05C505CD05D505000024003300A1
:101700003E004A005200DD05EC05F50504060D0615
:101710000000240033003E004A0052001C062A0646
:10172000340645065606FF010707FA050303FA04C7
:10173000010120000303FB040101FB0301011E045E
:10174000070738000707FB0601012E000101FA0216
:1017500003021D00FFFF1E000101FB050101300017
:101760000303300203031700FFFF1900FFFF3007D8
:101770000101360003021F0007040B00FFFF0700F2
:10178000FFFF0900FFFF0D00FFFF0F00FFFF01003B
:10179000FFFF0300FFFF0500FFFF00000000000047
:1017A00000001700FFFF1800FFFF1900FFFF1A00DD
:1017B000FFFF3A0701011E0103031F040302280073
:1017C0001F101B00FFFF1C00FFFF31001F162F061C
:1017D0000101270007043700010128070101220049
:1017E000070423007F5424007F5425000F0826009F
:1017F00007040E0001010F000F0010000F08110078
:101800000F0812000F0813000F0114000F0D150030
:101810000F0D16000F0D1F0301012B00FFFF2C0001
:10182000FFFF2D00FFFF300601013200FFFF3004F3
:101830000101300501013300FFFF3400FFFF3500D7
:10184000FFFF400000004100000042000000430094
:101850000000440000004500000046000000470072
:1018600000004800000049000000290001011B00A1
:10187000FFFF290101011D00FFFF290201010000F6
:1018800000003900FFFF00000000000000002A00F7
:10189000010132003400360090009200DE00E000CA
:1018A000A401A601A801AA01AC01AE01B001B201D8
:1018B000B401B601B801BA01BC01BE01C001001BF0
:1018C00077403E000102FFFF001E84803C000102C1
:1018D000FFFF003567E03E00FFFFFFFF0035C988CE
:1018E0003EFF010203040036EE803CFF01020304C8
:1018F000003875203EFF01FFFFFF0039FBC03EFFAF
:10190000FF02FFFF003D09003C000102FFFF005104
:1019100056443D000102FFFF005194C43D00010206
:10192000FFFF0051E2E43D000102FFFF0051F66CB1
:101930003D000102FFFF0052736C3D000102FFFFFA
:10194000006ACFC03E00FFFFFFFF006B31683EFF23
:1019500001020304006CB8083CFFFF020304006DA1
:101960007B583EFFFF02FFFF006F63A03C000102B7
:10197000FFFF009A1D203E000102FFFF009AE07069
:101980003C000102FFFF00D59F803E00FFFFFFFFEC
:1019900000D601283EFF0102FFFF00D7E9703CFF9F
:1019A0000102FFFF00D84B183EFF01FFFFFF00D9E7
:1019B0000E683EFFFF02FFFF00DAF6B03C000102B6
:1019C000FFFF0113B2203E000102FFFF011538C0E6
:1019D0003C000102FFFF01406F403E00FFFFFFFFA0
:1019E0000140D0E83EFF0102030401437C803CFF3C
:1019F000010203040143DE283EFF01FFFFFF014413
:101A0000A1783EFFFF02FFFF01474D103C0001029D
:101A1000FFFF017BCA903E000102FFFF017D5130B4
:101A20003C000102FFFF01AB3F003E000102FFFF4F
:101A300001B2E0203CFFFFFF030401C52FA03C00E2
:101A40000102FFFF06FD91D806FE300606FE718BEF
:101A500006FE300606FD91D806FCF3AB06FCB22666
:101A600006FCF3AB189518951895189518951895C8
:101A700018951895189518951895189518951895FE
:101A800018951895189518951895189518951895EE
:101A90001895FFB60F931F932F930091CD0300234A
:101AA00041F410E20E944E3311E005FD1FEF109348
:101AB000CD032F911F910F91FFBE1895FFB60F9385
:101AC0001F932F930091CC03002341F410E20E9456
:101AD0004E3311E004FD1FEF1093CC032F911F91A3
:101AE0000F91FFBE1895FFB60F921F920F931F9391
:101AF0002F933F93AF93BF93CF93DF93EF93FF93D6
:101B0000A0919E02B0919D02109729F01197A09389
:101B10009E02B0939D020091A002002319F00A9545
:101B20000093A0020091C80407FF0E94ED300091CD
:101B30005B02002361F00A9541F400915A020023F0
:101B400031F022240E94ED3002C000935B0200912C
:101B5000110407FF17C010911204112399F406FD18
:101B600003C00027112707C0109113041A9532F4FF
:101B700010E2012714E62CE02093120410931304C2
:101B80000093110400911004002319F00A950093AA
:101B900010040091000400230AF069C0A091F7032B
:101BA000B091F6031197A093F703B093F60309F0F1
:101BB0005EC00091FE030093F6030091FF030093C3
:101BC000F7030091CF04002309F011C00091CB046A
:101BD0001091CE0403951395011711F40091CD04D3
:101BE0000093CB040E94A7340E94314340C010E010
:101BF0000E941F34302F31702D911D910C91AF93A5
:101C0000BF931090F8030090F903000E111E00E03E
:101C1000201F301F31703F932F931F920F9211E0BE
:101C20000E941F34302F31702D911D910C910F9017
:101C30000016002D0F900106102D0F900206202D8A
:101C40000F900306302D49F044F03091FA032091B3
:101C5000FB031091FC030091FD03BF91AF910C9326
:101C60001E932E930E910E7F3170302B3C93B091CA
:101C70000208A09103081097B1F01197B0930208E1
:101C8000A093030881F40FEF009327020093DE0373
:101C90000093C6030093510300938B0200936402E8
:101CA00004E100934701B0919906A0919A0610971C
:101CB000C1F01197B0939906A0939A0691F4F4E0BD
:101CC000EAEAAA27BB27D1E0C1EE0E949730102F85
:101CD0000081011711F00E949E30119631962197D4
:101CE000A1F7B0919B06A0919C06109761F0119707
:101CF000B0939B06A0939C0631F40FEF0093AC02C7
:101D000001E000939003B091F203A091F3031097C8
:101D100049F01197B093F203A093F30319F401E093
:101D20000093F00300915802023321F003950093D1
:101D3000580209C000915A02002329F401E00093DF
:101D40005A020E94ED303FEF00915302002359F0F8
:101D50000A9500935302002399F410E20E944E3337
:101D6000009336010DC010E20E944E3302FF05C001
:101D700003FF03C00093360103C002E30093530244
:101D800000919806002319F00A9500939806009197
:101D9000320110913301011709F058C0009134014C
:101DA0000F7B109135011F7B011731F066240091E4
:101DB00034010074102BDDC000912902002319F0BA
:101DC0000A950093290200912D01002309F010C10A
:101DD00011270E944E331091A80210FD0F7710FDBD
:101DE00010951093A80210915802113319F00F3F6B
:101DF00009F462C01091F00317FF11681093F0030B
:101E00001091320120E80090D00110909A01012831
:101E100010909901012800FC006810FC006407FF85
:101E20001227269506FF1227269505FF12272695CD
:101E300004FF1227269503FF1227269502FF12277B
:101E4000269501FF1227269500FF122700913201E7
:101E5000012706FF02C016FD3E7F3093050407FFF1
:101E60000AC0009134010C70C9F421E017FF2FEF74
:101E70002093CB0113C004FF11C030910C040091DA
:101E80000E0404302CF414FD316014FF3E7F04C0B6
:101E900014FD306814FF3F7730930C041093320127
:101EA0001093330110955090370110933701012F93
:101EB00010E30E944E339BC010E10E944E33202F4E
:101EC0000074109134011F7B012B00933401022F09
:101ED0000F7B3091050410FF03233FEF309305047F
:101EE0001091A90210FD0B7F10FD10951093A9020F
:101EF0001091AA0210FD077F10FD10951093AA0201
:101F000010919B0110FD0E7F10FD109510939B0109
:101F100010915802113319F00F3B09F46CC0109165
:101F2000F00317FF11681093F0031091340120E8BB
:101F300066240090D00110909A01012809F00C61EC
:101F40000090990100FC016007FF6094269526959A
:101F500005FF1227269504FF1227269503FF122757
:101F6000269502FF1227269501FF1227269500FFCE
:101F700012271093340110933501109550903A01B7
:101F800010933A01012F10E60E944E33662019F09B
:101F90002FEF2093C3020091C804087041F500910F
:101FA0003A010525087029F001E053FE0FEF009378
:101FB000C70100913A010525047029F001E052FEA5
:101FC0000FEF0093C90100913A010525027079F0E5
:101FD00051FE03C00E94722E07C0002700939B068B
:101FE00000939C060093AC020FEF0093900306E968
:101FF0000A9500932D01009151020023B9F400913C
:102000003601007410915202102710E069F010E2BE
:102010000E944E33202F00740093520211E0207C66
:1020200011F0203C09F41FEF1093510200EE06BDA1
:10203000FF91EF91DF91CF91BF91AF913F912F91A0
:102040001F910F911F900F90FFBE1895FFB6AF9391
:10205000BF930F931F932F930091A506002319F0B0
:102060000091C60031C0B6E0A7EA1091A60600278D
:10207000A10FB01F0091C600003234F10C931395EC
:102080002091E1042223A1F0163440F02091A50212
:1020900020FD0EC021682093A5020AC01A3040F42A
:1020A0002091A50220FD04C02E7721602093A50277
:1020B000103511F01093A6060B3331F40FEF009397
:1020C000A50600270093A6062F911F910F91BF919F
:1020D000AF91FFBE1895FFB6AF93BF930F931F93B9
:1020E0000091F706002331F40091C1000F7D0093A9
:1020F000C1000EC0B6E0A9EF1091F806101B0A95BA
:102100000093F7060027A10FB01F0C910093C600A3
:102110001F910F91BF91AF91FFBE1895FFB60F921F
:102120001F920F931F932F933F93AF93BF930091F1
:10213000DA04007161F10091340106FF28C0EF93C9
:10214000FF93FAE1E4E411270091E803000F111F67
:10215000000F111FE00FF11F05910093DF030591A0
:102160000093E00305910093E10304910093E203DF
:10217000FF91EF9120E10E944D2D0E94AB2D009127
:10218000E8030395083009F400270093E803009161
:102190002C010C3019F41FEF1093A702083019F42A
:1021A0003FEF3093A402302F000F1127ACE8B4E0CA
:1021B000A00FB11F009178001091790011963F9304
:1021C000373084F411971D900C90332723E0200DB5
:1021D000311D0217130734F49001225030400217CA
:1021E000130714F40C931E933F9133953F3021F461
:1021F00033270FEF0093AF0230932C0107E0301725
:102200000CF4032F00937C0000913801087F132FFA
:1022100017501770012B00933801086010E40E94DA
:102220004E330FED00937A000091DA04007109F04B
:1022300046C000910E040A3009F041C000913401FB
:1022400006FF3DC001EC0E949E330091380110E46E
:102250000E944E330FEF08B9002707B90E94B6332A
:10226000009311010E94B6330093120110911101E5
:1022700000911201000F111F000F111F000F111FFD
:102280009801000F111F020F131F20E030E010F41F
:102290002FEF3FEFB8ED0B0FB1E91B1FBDEF2B1F69
:1022A000B6E03B1F3093DF032093E0031093E1037C
:1022B0000093E20320E10E944D2D0E94AB2DBF91BF
:1022C000AF913F912F911F910F911F900F90FFBEE3
:1022D0001895FFB620905A02222089F00F921F9283
:1022E0000F931F932F93EF93FF9322240E94ED30BF
:1022F000FF91EF912F911F910F911F900F90FFBEB3
:10230000189500E10EBF0FEF0DBF00E002B90027E6
:1023100001B90EE405B90093300103EF04B90FEFE2
:1023200008B9009507B90FE00BB90093310102EF2E
:102330000AB9A0E0B1E0E8E6F8E0EA1BFB0B0027F1
:102340000D933197E9F70FEB009334010FEF0093F2
:10235000320100933A010093EB030093250101E061
:1023600000938402009328020FE700939D060AEA77
:1023700000938C0400938D0400E8009338010093CF
:10238000F00308E0009339010AE000937F02009314
:102390008202E8E5F5E0A8E4B1E005E10E9401343D
:1023A000EEE6F5E0ADE5B1E007E20E940134EAEBCC
:1023B000F5E0ACE9B1E00DE00E940134E8E0F6E0C0
:1023C000A4E8B1E00DE00E940134E6E1F6E0A0EB04
:1023D000B2E00DE00E940134EEECF4E0A4ECB2E0D7
:1023E0000EE00E940134E0ECF4E0A6E2B3E00EE07F
:1023F0000E940134EEE3F6E0A4E3B3E007E10E94BB
:102400000134ECEDF4E0A3E5B3E00CE00E9401340C
:10241000E2E3F6E0AEE6B3E00BE00E940134E6E56D
:10242000F6E0A1E9B3E00FE00E940134E6E6F6E051
:10243000A0EAB3E007E10E940134EAEBF6E0A9EB81
:10244000B3E00CE00E940134E2E3F7E0A9EEB7E06C
:102450000CE00E940134EAE1F7E0A5E0B8E007E112
:102460000E94013400913901016010E50E944E3351
:10247000009139010E7F10E50E944E3304E11DE109
:1024800028E20E94CA3304E11DE120E20E94CA331F
:102490000AE41EE128E20E94CA330AE41EE120E2B7
:1024A0000E94CA3300271FE128E20E94CA33002796
:1024B0001FE120E20E94CA3300E410E228E20E94F9
:1024C000CA3300E410E220E20E94CA3301E020E1B6
:1024D0000E94833301E028E30E94833301E020E37C
:1024E0000E94833301E028E10E9483330E94AB2DD8
:1024F000002707B9009508B9F4E0EAEAD1E0C1EE97
:10250000BB27AA270E949730019311962197D1F7F4
:102510000E94A73400270093D404332722271127D1
:102520000091CB045FEF48E00E94AF2D0091B8010D
:1025300000937A030093E6030091B90100937B03B3
:102540000093E70311270091C80403FD10E81093DE
:10255000330110E00E941F340E7000930D04102F01
:102560000091C80403FD1091AB041E7010930E047B
:1025700011270091B70407FD18E000FD14601093C7
:1025800035010E94303403701127002339F012E026
:10259000013021F011E0023009F013E01093330113
:1025A00000E300930F040AE00093F50308E00093B2
:1025B00091060CE4009392060BE40093930600E46A
:1025C00000939406002700939506009396060091C9
:1025D000D20400780093EF0391F404E100934701E3
:1025E0000FEF009327020093DE030093C6030093CE
:1025F000510300938B020093640200930504009141
:10260000DF0415E0019F800123E033270E94874308
:1026100000930A04109309040091DA040C700093EB
:10262000F103BB27AA27002351F0BDEDA0ED043034
:1026300031F0BBEBA0EA003111F0B7E7A0E4B093B2
:10264000F203A093F30303E000937C000CED0093EE
:102650007A0000270093C5001091D10407E61123EA
:1026600051F003E3113039F009E1123021F000E1BB
:10267000133009F008E00093C40008EB0093C10098
:1026800006E00093C2000091E104002319F001E884
:102690000093A50200EE06BD05E005BD01E0009334
:1026A0006E000FE30093690007E00DBBB3E0A8EEF6
:1026B0001B9902C01197E1F700913801086010E4FE
:1026C0000E944E3300270E949E330E949E330E9438
:1026D0009E330E949E330E949E330E949E330E942E
:1026E0009E330E949E330E949E330E949E330AEACC
:1026F0000E949E330091380110E40E944E330FEF88
:1027000008B9002707B90E94B633053529F00CE156
:1027100000935D0200935E02789400915E020023B4
:1027200009F0FACF0091AF020023B1F300919F02AC
:10273000002381F40091D4040023A9F0F8940FEF52
:1027400000939F02B3E1A8E8B0939D02A0939E027C
:10275000789409C0F894B0919D02A0919E021097C0
:1027600011F40C94007E0091EF030023E9F0009136
:1027700004081091EB03012BB9F4B7E0A9E4F7E0EA
:10278000E5EF1CE00D9101931A95E1F7B9E0A4EC97
:10279000F894B0930208A0930308789408E100939A
:1027A00001080FEF00930408F894209138012F7B63
:1027B00010E40091D90400740127022B0093380122
:1027C00078940E94453500918F030023D9F44091FD
:1027D000900340FF17C00CE41FE623E63BE647FFEB
:1027E00003C000E2102F980100939C0310939D03F7
:1027F00020939E0330939F030FE000938F030027E5
:1028000000939003009100040023FAF40091220049
:1028100017E1019F02E7000D1091A9041017A8F01D
:10282000F89400270093F6030093F70303950093B1
:1028300000042091AE0204E516EA0E94E82F2091E0
:10284000AD0204E515EA0E94E82F0091F00300FFB5
:10285000AFC00E7F0093F00307FF60C00FEF00933F
:10286000C80305E00093C7032091AE0204E516EA11
:102870000E94E82F2091AD0204E515EA0E94E82F9E
:1028800000919A020093E20404E11DE128E20E9413
:10289000CA3304E11DE120E20E94CA3301E020E1D5
:1028A0000E94833301E028E30E94833301E020E3A8
:1028B0000E94833301E028E10E9483330E94AB2D04
:1028C0000091410110EC0E946A3300913B0110E736
:1028D0000E946A330091420110ED0E946A332091F8
:1028E000E50410E50EE90E94E82FBB27AA27009116
:1028F000DA040C700093F10351F0BDEDA0ED04304B
:1029000031F0BBEBA0EA003111F0B7E7A0E4F89496
:10291000B093F203A093F30378944AC00027009386
:10292000C80305E00093C703222704E516EA0E94C6
:10293000E82F222704E515EA0E94E82F0091E2041F
:1029400000939A0200270093E20407E128E20E9424
:10295000CA3307E11DE120E20E94CA3304E020E10E
:102960000E94833304E028E30E94833304E020E3E1
:102970000E94833304E028E10E9483330E94AB2D40
:10298000009141010C7F10EC0E946A3300913B01E1
:102990002B7F10E70E946A330091420100640F7D93
:1029A00010ED0E946A332FEF10E50EE90E94E82F28
:1029B0000091C6030023F9F00091C5030023D9F468
:1029C00000270093C60300910004002311F003E5E3
:1029D0000DC000910104002311F00DE407C0009127
:1029E000AA040550F2F70A5F10E3010F0093C40335
:1029F0000CE00093C503309187020091A7020023E9
:102A000009F473C0F89400270093A7021091A4045E
:102A10000091A504789416950795169507950C3D99
:102A200008F063C0033C30E098F431E0053A80F4EC
:102A300032E0073868F433E0093650F434E00B3400
:102A400038F435E00D3220F436E00F3008F437E08A
:102A500030938702363099F000910804002309F082
:102A600044C0002700930604EAE1F7E0A5E0B8E0DF
:102A700007E10E94013407E10093080436C03430B6
:102A800041F000910004002321F00027009300048E
:102A90000BC0353051F100910104002331F10027C2
:102AA000009301040E94064410E00E941F343091FC
:102AB000FA033E933E7030930D040091C80403FF67
:102AC00030930E042091FB031091FC030091FD0351
:102AD00011962D931D930C930FEF0093C603009353
:102AE00051030093DE03009327020091C3020023E9
:102AF00009F4F9C000270093C3020091D00100231C
:102B000009F0DCC03091870234300CF4C5C0343099
:102B100009F41DC0353009F4A0C0363009F0E3C017
:102B200000910604002341F4009107040E943144FF
:102B30000FEF00930604D7C000910E0404300CF090
:102B4000D2C00091070403950093EE03CCC0F89423
:102B5000009100040095009300048AF001E00093C6
:102B600000042091AE0204E516EA0E94E82F2091AD
:102B7000AD0204E515EA0E94E82F7894B4C00E3F38
:102B800071F010E00E941F340093FA030D9100933E
:102B9000FB030D910093FC030D910093FD037894CA
:102BA0000091CF04002309F00BC0F8940091CD04EC
:102BB0000093CB0478940E94A7340E94314323C031
:102BC0000091CF0422271AE00130C9F014E6023048
:102BD000B1F023E018EE033091F027E210E1043069
:102BE00071F02AE318E9053051F02EE410E20630C6
:102BF00031F021E618EA073011F023EC10E52093BC
:102C0000F8031093F9030091D004222712E3002364
:102C100061F01DE7013049F01AEF023031F021E098
:102C200014EF033011F029E014ECF8942093F6032C
:102C30001093F7032093FE031093FF037894222749
:102C400004E516EA0E94E82F222704E515EA0E940F
:102C5000E82F0FEF0093C60346C010E00E941F3418
:102C60000093FA030D910093FB030D910093FC0375
:102C70000D910093FD0300910104002319F00E94BF
:102C8000314331C00FEF009301040093C6030E944B
:102C9000A7340E94DA3427C000914C0200950093BB
:102CA0004C020AE210E211F000E21AE200933F0344
:102CB000109348030FEF0093510315C00091CF010B
:102CC0000D3011F00E3079F41091D10116305CF016
:102CD0000091EC0303950C3009F400270093EC03FA
:102CE0000FEF0093E9030091340106FF06C00E9434
:102CF0009E450E94BC450E942046F89410919E0477
:102D000000919F047894000F111F00930C01109301
:102D10000B010091C8040670043029F0063019F048
:102D20000027112714C0F8941091A6040091A7045D
:102D30007894000F111F000F111F000F111F000FBB
:102D4000111F000F111F33272AE00E9487430093B1
:102D5000080110930701F8941091A0040091A104B8
:102D600078941695079500930A0110930901F89439
:102D70001091A2040091A304789416950795222738
:102D800033274091C804542F40774032D9F456700D
:102D90005630E1F013E300916902109F8001332760
:102DA00020916402222309F423950E948743073669
:102DB00008F007E600936C033327222714E6019FEF
:102DC000800104C0202F312F00271127009310010C
:102DD00010930F0120930E0130930D0122270091D3
:102DE000340106FD206800910E0404300CF02064CC
:102DF00000910C0400FD206200913A0105FF206162
:102E00000091C904007306950695202B1091CA0401
:102E10001370212B2093A602209139012971009172
:102E2000E4040078202B0091F003009500780695CB
:102E30000695202B00919902202B1091250111233A
:102E400021F410913901211741F0F89420933901B0
:102E5000022F10E50E944E3378940091C80406704A
:102E600009F4DAC100918D022091C204109125016C
:102E7000112311F4021731F020938D0212E008E5BE
:102E80000E94E82F22270091DA0407FD2FEF00911E
:102E90000E04083009F42FEF00912501002321F4DE
:102EA00000919302201731F02093930211E008E57E
:102EB0000E94E82F0091C8040078B9F0F8941091AE
:102EC000900420919104789416952795169527954E
:102ED00000912501002391F430917302231729F00A
:102EE000209373020027009375020091750200FD84
:102EF0002091740200917202021731F02093720245
:102F0000112708E50E94E82F20917C020091C80457
:102F1000007851F0F89430919804209199047894B5
:102F20003695279536952795369527953695279585
:102F30003AE7230F0091DA0405FF05C02093E60469
:102F40000E94063420C000912501002391F40091D5
:102F5000C804007849F030917B02231729F02093B0
:102F60007B02002700937D0200917D0200FD2091ED
:102F70007C0220937A0200917A02021721F016E572
:102F80000EE90E94E82F00910E040430A4F00A30EC
:102F900091F0083081F02091DC040091250100239C
:102FA00021F400918502201731F02093850214E569
:102FB0000EE90E94E82F209167020091C804007872
:102FC00051F0F894309196042091970478943695B6
:102FD0002795369527950091DA0405FF0BC02195BA
:102FE0002A3F10F4263308F4F7C02093E5040E942A
:102FF0000634F2C026951091C804107849F010915B
:103000006602121729F020936602112710936802B6
:103010001091680210FD209167020091640202176E
:1030200029F400912501002309F430C020936402A3
:103030000091C102002351F546E00091C8040670DA
:1030400019F0023009F047E033272227009164028B
:103050001AE0019F800155270E94AF2DADEBB2E031
:103060000091B6010D930091B7010D930091B80145
:103070000D930091B9011091C804167019F0123027
:1030800009F000E20C9301E10093C10200913401C8
:1030900006FD04C0002700936902BEC00091DA0457
:1030A00006FF9AC000910E04003029F0023019F09A
:1030B0000A3009F01CC0F89400913801086010E44F
:1030C0000E944E3305EC0E949E330091380110E4BB
:1030D0000E944E330FEF08B9002707B90E94B6339C
:1030E0007894002321F400270093690295C0109181
:1030F000A302112319F0123009F08EC000270093AB
:10310000A302109121010091220133272AE040916E
:10311000C804467019F0423009F024E60E94874343
:10312000009369021091640216C0309169033A510C
:1031300090F041E1349F80012AE033270E948743C9
:10314000109164023FE7301B37FD3327009169027D
:10315000311708F4132F21E0101B19F40093A20279
:103160005BC010F4119521953091F503131718F4F5
:103170000093A20251C000270093A2021091E5041F
:10318000121B1A3F68F4163328F01093E5040E94CE
:10319000063422C019EF1093E5040E94063405C0DE
:1031A00016E31093E5040E9406341091E604120F12
:1031B0001A3B68F41A3728F01093E6040E9406348C
:1031C0000BC019EB1093E6040E94063405C01AE701
:1031D0001093E5040E940634442700919C0220913C
:1031E000E604021739F020939C0212E50EE90E94D2
:1031F000E82F4FEF00919B022091E504021739F070
:1032000020939B0210E50EE90E94E82F4FEF442324
:1032100019F001E00093A302789400910D040A30A4
:1032200011F420EC3FC00091C8040078C1F0F8947C
:103230001091920400919304789498013695279503
:103240003695279530917702321729F0209377022F
:103250003327309379023091790230FF07C011276C
:1032600000917802000F111F000F111F109500959B
:1032700013702BEE35E0020F131F2091D504332776
:10328000220F331F220F331F220F331F220F331F32
:10329000200F311F3695279536952795369527951A
:1032A000369527950091C904087029F400913401DE
:1032B00006FF01C020EC0091760210912501112338
:1032C00011F4021731F02093760214E10EE90E9406
:1032D000E82F0091C804007899F0F8943091940494
:1032E00020919504789436952795369527953091B9
:1032F0006F02231729F020936F02002700937102B9
:103300000091710200FD2091700226952695269568
:1033100000912501002321F400916E02021751F063
:1033200020936E0200E515EA0E94E82F00E516EAF8
:103330000E94E82F0091C804007899F0F894309129
:103340008E0420918F04789436952795369527958D
:1033500030916B02231729F020936B020027009312
:103360006D0200916D0200FD20916C02269526955C
:10337000269500912501002321F400916A0202178D
:1033800051F020936A0202E515EA0E94E82F02E557
:1033900016EA0E94E82F789411270091370102FF66
:1033A00013C003FF22C02091AE02222321F42FE19B
:1033B0002093AE021FEF2091AD02222331F52FE1C1
:1033C0002093AD021FEF21C02091AE02222321F0F5
:1033D00022272093AE021FEF2091AD022223A9F0F5
:1033E00022272093AD021FEF10C02091AE022223AE
:1033F00021F42FE12093AE021FEF2091AD02222392
:1034000021F022272093AD021FEF00912501002318
:1034100011F4112361F02091AE0204E516EA0E9436
:10342000E82F2091AD0204E515EA0E94E82F2091D3
:10343000C804207899F0F89430918C0420918D0480
:103440007894369527953695279530916102231704
:1034500029F0209361020027009363020091630228
:1034600000FD2091620200912501002349F40091A2
:1034700060021091630210FD00916202021731F0A8
:103480002093600216E10EE90E94E82F78942091C3
:103490008702222329F44091510240935203CFC066
:1034A00024300CF47AC0243009F443C0253009F1EB
:1034B000263009F0C4C00091070410915102112375
:1034C00031F032F40A95002342F409E006C0B7C097
:1034D000102F03950A300CF00027109108041123D7
:1034E00021F4009307040E94314400270093510205
:1034F000A6C0F8940091CB0410915102112339F029
:103500003AF40F770A9500234AF404E507C097C000
:10351000102F0F77039505350CF000270093CB048F
:1035200078940E94A7340E94DA3400270093510255
:1035300086C0F8940091D00410915102112389F0B3
:103540002091D001222309F023C0112322F40A95EF
:103550004AF4002707C00395043024F019F004E072
:1035600001C06DC00093D004222712E3002361F054
:103570001DE7013049F01AEF023031F021E014EF7D
:10358000033011F029E014EC2093FE031093FF03A5
:10359000002700935102789452C00091C202002388
:1035A00009F04DC040914C0200915402442311F0A7
:1035B0000091550240915102442329F012F00395E5
:1035C00009C00A9507C02091560227FF38C02F77FF
:1035D0002093560212E3213021F014E6223009F044
:1035E0001AEF002372F40C3E0AF40CEE0195019FD1
:1035F0000094109411E0010E10E0111E1FEF0195D0
:1036000005C005310AF004E1019F112740914C02E9
:10361000442359F4009354021093D6031093D70314
:103620001092D8030092D9030AC000935502109358
:10363000DA031093DB031092DC030092DD030E9497
:103640003034212F1C7116951695312F00910D04E1
:10365000083009F430622076203039F0203419F037
:10366000203639F007C0386005C004301CF03860DF
:1036700001C030611091C904187009F030641091D4
:10368000C804117009F0306800912501002321F46D
:1036900010913D01311731F030933D01032F10E9B6
:1036A0000E946A3320EA00910D040A3019F42F7D3C
:1036B000206500C0009152030023B1F01091500228
:1036C00040914C0240FF10914F02010F12F403E0B1
:1036D00003C004300CF00027442319F0009350027B
:1036E00012C000934F020FC010E00E941F34007FF1
:1036F0000295102F037000934F02012F0695069537
:103700000370009350021FE000914F02100F0E94BF
:103710000D34083031F4002700934F021FE00E945F
:103720000D34332710914D02101719F03FEF00931D
:103730004D021AE0019FECE7F0E0E00DF11D359637
:10374000A2E4B3E005910D9305910D9305910D93BE
:1037500005910D931596BF93AF933F9313E100919D
:103760005002100F0E940D340D3031F400270093E9
:10377000500213E10E940D343F9110914E02011747
:1037800019F03FEF00934E02AF91BF911AE0019FF5
:10379000ECE1F2E0E00DF11D359605910D930591F8
:1037A0000D9305910D9305910D9300915103032BFA
:1037B00051F000915003002331F40CE100935003C9
:1037C00000270093510300915002000F000F109149
:1037D0004F02102B1F9300915203002399F00027F2
:1037E0000093520310E00E941F340F701F911F932B
:1037F0001295012BF8940E930E94063478940FEFE3
:103800000093DE031F91212B00912501002321F459
:1038100010913E01211731F020933E01022F10EA52
:103820000E946A330091C202002309F071C0009126
:10383000370106FF6DC000915102002321F00027DF
:103840000093510208C00091DE03002309F460C018
:1038500000270093DE0340914D020AE2409FECEC0A
:10386000F0E0E00DF11DA2EDB2E00AE20E940134A9
:1038700040914E020AE2409FEEE9F2E0E00DF11DB8
:10388000ACEFB2E00AE20E940134009154021091C0
:10389000D802100F1093D8021091DC02100F109371
:1038A000DC021091E602100F1093E6021091EA027A
:1038B000100F1093EA021091F402100F1093F4020B
:1038C0001091F802100F1093F80200915502109118
:1038D0000203100F1093020310910603100F1093B0
:1038E000060310911003100F10931003109114038E
:1038F000100F1093140310911E03100F10931E034A
:1039000010912203100F1093220300E70093C202CC
:1039100000918E030023E1F41091C80410771295F2
:1039200000912501002329F400918B02011709F46D
:103930000FC010938B020AE0019FF4E0E8EEE00D67
:10394000F11DB3E0AFE50E94013406E100938E0360
:103950000091C8040077003009F41EC0003109F45A
:1039600022C0003209F42DC0003309F42DC0003408
:1039700009F42DC0003509F42DC0003609F42DC01E
:10398000F8941091A0040091A10478942CE33327BB
:103990000E948743202F37C0F89410919E04009115
:1039A0009F0478942BC0F8941091A2040091A30472
:1039B00078942AE033270E948743202F00936D03D9
:1039C00022C020916C031FC0209169031CC020916C
:1039D0006A0319C020916B0316C0F8941091070177
:1039E00000910801789416950795169507951695F8
:1039F0000795169507951695079500C02AE0332779
:103A00000E948743202F00912501002321F400917B
:103A10008A02021731F020938A0210E10EE90E9417
:103A2000E82F0091C804067009F404C100910E0447
:103A3000222704302CF008303CF071F00A3011F4E9
:103A4000206811C028690FC020610E9430340072C4
:103A500009F02068286007C020620E94303400729C
:103A600009F0206828601091C8041670163009F417
:103A70002460216000910E04003051F0023041F0CA
:103A8000083031F00A3021F010910C0417FF2E7F1E
:103A90002F930E943C343E91317011962D911D91CF
:103AA0000C9170E06EE154E840E80E94F4332F91ED
:103AB0000CF422600091C8040077003209F42064FD
:103AC00000912501002321F410913B01121731F0E0
:103AD00020933B01022F10E70E946A330E943C347E
:103AE0003E91317011962D911D910C918827409136
:103AF0003B0141FD1CC070E06BE55DE840E80E94C1
:103B0000F43314F4806113C070E067EB5BE140E0D4
:103B10000E94F43314F480620AC071E061E35DE254
:103B200040E80E94F43314F4806401C0806870E0BF
:103B300066E255E240EA0E94F43314F421E049C001
:103B400070E06CE45BE440E40E94F43314F422E09F
:103B500040C070E063E55CEE40E60E94F43314F48C
:103B6000222737C070E062E750E740EE0E94F4334E
:103B700014F423E02EC070E067EB5BE140E00E94AC
:103B8000F43314F424E025C070E064EF54E240E024
:103B90000E94F43314F425E01CC071E061E35DE29F
:103BA00040E00E94F43314F426E013C071E06FE4A7
:103BB00051EB40E80E94F43314F427E00AC071E0AE
:103BC0006BEA5FE340E00E94F43314F428E001C0A4
:103BD00029E0822B00912501002321F410913C0162
:103BE000811739F080933C01F894082F10E80E9467
:103BF0006A338695869586958E7109F48160806416
:103C00000091C804067021F0023011F080628F7BB1
:103C10000091F0030078802B00912501002321F40E
:103C200010914201811731F080934201082F10ED6D
:103C30000E946A330E943C34222713960C9108702C
:103C400009F020683FE744270091320105FF61C079
:103C5000822F0E911E912E913E913170110F221FD5
:103C6000331F442755276EE1B4E0A4E10EE1061BA3
:103C7000000F000F1127A00FB11F1D9117FD04C0E9
:103C800050FF962F5FEF11C013700D9102171307AD
:103C900061F40D911C91712F782777FD06C04FEFCD
:103CA00000939E061F7710939D066A95E9F650FFD4
:103CB0009EE10091340106FF27C00091D30402FF6A
:103CC00004C00B7F0093D30402C04423E9F42F9374
:103CD0003F938F939F930E947C449F918F913F913C
:103CE0002F91B4E0A4E10EE1091B000F000F112792
:103CF000A00FB11F30683D932D9300919E060D9348
:103D000000919D06082B0C93282F30919D06409121
:103D10009E0664E057EA46FD02C05A50604045FDE9
:103D200002C05451604044FD02C05752604043FD00
:103D300002C05255604042FD02C05659604041FDEC
:103D400002C05A54614040FD02C05053624060932B
:103D50001B0150931C010091D3040D7F47FD0260AD
:103D60000093D30466E258EE36FF02C0565160401D
:103D700035FF02C05253604034FF02C05A586040C1
:103D800033FF02C05652624032FF02C0585D6440A9
:103D900031FF02C05E566A4030FF02C05A5A644189
:103DA00060931D0150931E01232B009125010023D8
:103DB00021F410914401211731F020934401022F86
:103DC00010EF0E946A33242F00912501002321F473
:103DD00010914301211731F020934301022F10EE7F
:103DE0000E946A3380E100913701037049F002308C
:103DF00029F0013039F484608F7E04C0816001C0F5
:103E0000836080620E9430340C7F1127803139F04A
:103E10001395843021F01395813309F01395012B0C
:103E20000E93007109F080641091C904187009F0B4
:103E3000806410E00E941F34302F31702D911D914D
:103E40000C9170E069E150EF40EA0E94F4330CF00D
:103E5000806800912501002321F410914101811710
:103E600041F0809341010E940634082F10EC0E941B
:103E70006A332091D70400913D01007211F4209122
:103E8000D60400912501002321F400918902021734
:103E900031F02093890212E10EE90E94E82F0E947E
:103EA0003034007419F080E89FE76AC088279FEFDC
:103EB00010E00E941F34302F31702D911D910C9114
:103EC00070E06BE157E740E40E94F43314F49B7F09
:103ED00057C070E06DE256EC40EC0E94F4331CF4E5
:103EE00084609B7F4DC070E06DE359E040E00E942C
:103EF000F43314F4977F44C070E066E65FEF40E36C
:103F00000E94F4331CF48860977F3AC070E069E83F
:103F100054E540E40E94F43314F49F7E31C070E015
:103F200060EA57E340EA0E94F4331CF480619F7E0C
:103F300027C070E06FEA59E740EE0E94F43314F4B2
:103F40009F7D1EC070E064EF54E240E00E94F433B5
:103F50001CF480629F7D14C071E061E35DE240E08B
:103F60000E94F43314F49F7B0BC071E06DE758E7B7
:103F700040E40E94F4331CF480649F7B01C09F776F
:103F800000912501002341F400913F01081721F41D
:103F900000914001091761F080933F019093400127
:103FA000082F10EB0E946A33092F10EB0E946A332E
:103FB00022270091C10410918C02011719F02FEFF4
:103FC00000938C020091C30410918E02011719F026
:103FD0002FEF00938E020091C40410918F020117FD
:103FE00019F02FEF00938F020091C50410919002F9
:103FF000011719F02FEF009390020091C604109161
:104000009102011719F02FEF009391020091C7045C
:1040100010919202011719F02FEF00939202009174
:10402000D2040F7110918802011719F02FEF00933D
:10403000880200917F0210917E02011719F02FEF84
:1040400000937E020091820210918102011719F003
:104050002FEF009381020091E20410919602011764
:1040600019F02FEF009396020091EE03002309F060
:104070002FEF0091A60210919402011719F02FEF73
:10408000009394020091E00410919502011719F039
:104090002FEF0093950200912501202B29F4009128
:1040A000EA03002309F477C0F8942F9300913801B4
:1040B000086010E40E944E330091EA03002369F087
:1040C0000AED0E949E3310EAD7E0C9E409910E94EC
:1040D0009E331A95D9F71093EA032F91222309F4FE
:1040E00050C005ED0E949E330091C1040E949E3392
:1040F0000091C3040E949E330091C4040E949E3329
:104100000091C5040E949E330091C6040E949E3314
:104110000091C7040E949E330091D2040F7111F0E8
:1041200014E0010F0E949E3300918002002311F0E1
:1041300000917F020E949E3300918302002319F0B8
:104140000091820203950E949E33009196020E9484
:104150009E330091EE03003839F402E00093EE0341
:104160000A950E949E3305C00E949E33002700934B
:10417000EE030091A6020E949E330091E0040E948B
:104180009E3378940091020810910308012B19F4D2
:1041900000270093250100910E040A3021F40091BC
:1041A000340106FD31C2F89400913801086010E432
:1041B0000E944E330091EB030023D9F004EC0E94DF
:1041C0009E330091380110E40E944E330FEF08B97E
:1041D000002707B910EAD7E0C9E40E94B633099373
:1041E0001A95D9F71093EB030E94B6330093E304BA
:1041F0006EC002EC0E949E330091380110E40E94D0
:104200004E330FEF08B9002707B90E94B633009369
:104210001F010E94B633009320010E94B633009321
:1042200015010E94B633009316012091C8042F7720
:104230001091150117FD20682093C8041F77109373
:10424000150127FD14C00FEF00936302009368026D
:1042500000937D0200936D0200937102009375023A
:1042600000937902009380020093830230C0309162
:10427000970220912001231791F020939702332772
:1042800030938002222309F423E114E003E90E9421
:104290008743F89400931A0100270093190178943A
:1042A00020911F0100919802021789F03327309363
:1042B000830220939802222309F420E21AE702E104
:1042C0000E948743F8941093170100931801789483
:1042D00010911501009116012091A5022F7B16FD6A
:1042E00020642093A5021F7326FF18C020FF16C06C
:1042F0002E7F2093A502F8941F930F93009138010D
:10430000086010E40E944E330FED0E949E3300912E
:10431000A5020E949E330F911F9178942091320143
:1043200026FD72C1169507951695079511E0013384
:1043300010F112E00134F8F013E00135E0F014E080
:104340000136C8F015E00137B0F016E0013898F0FA
:1043500017E0013980F018E0013A68F019E0013BFC
:1043600050F01AE0013C38F01BE0013D20F01CE069
:10437000013E08F0112700919806002309F044C17E
:1043800000919706002351F4112309F43DC11BE06D
:104390001093980603950093970636C1013039F4BF
:1043A0000091CC010130C9F0023059F0D2C0112384
:1043B00009F02AC11BE01093980600270093970686
:1043C00023C11B3009F417C11C3021F411271093AD
:1043D000CC0111C11093EE030EC1113031F400274E
:1043E0000093CC010E94064406C1123041F4F894B7
:1043F0001091340104E0102710933501FCC01330F4
:1044000041F4F8941091340108E01027109335011D
:10441000F2C0143041F4F8941091320100E81027F2
:1044200010933301E8C0153019F40E943143E3C002
:104430001730D1F4F89410E00E941F34302F00930D
:104440008B062D9120938C061D9110938D060D9156
:1044500000938E064D9140938F064C914F7E409372
:1044600090060E94DA34C7C0183051F5F89410E075
:104470000E941F34009191060E930E7000930D045C
:104480001091C80413FF00930E0411960091920638
:104490000D93009193060D93009194060D93009156
:1044A00095060D93009196060C930FEF009327024B
:1044B0000093DE03002700935402009355029BC033
:1044C0001930B1F4F89410E00E941F340093910663
:1044D0000D91009392060D91009393060D91009318
:1044E00094060D91009395060D910093960683C056
:1044F0001B3089F4F8940091CB04102F0F770395AB
:1045000005350CF00027F8940093CB040E94A734E3
:104510000E94DA3470C01A3041F4F89410913201DC
:1045200008E010271093330166C01C3009F063C007
:10453000F8940091CB04102F0F770A9500230AF40A
:1045400004E5F8940093CB040E94A7340E94DA3467
:1045500052C0113011F4002735C0123011F405E0BB
:1045600031C0133011F40FE02DC0143011F404E108
:1045700029C0153011F409E125C0163011F40EE1FF
:1045800021C0173011F403E21DC0183011F408E205
:1045900019C0193011F40DE215C01A3011F40AE0F7
:1045A00011C01B3021F402E00093CC0124C01C3068
:1045B00011F501E00093CC01F8940E94A7340E9409
:1045C000DA3419C0402F4B5F0093AA040E943034A4
:1045D00017FD05C00091AA0403950417A9F70FEF72
:1045E0000093C6030093DE03009327020027009385
:1045F0005402009355020091970603950093970685
:10460000F8940E94063478940091CE03002369F553
:1046100011271093CE030091CC0300FF26C0109306
:10462000CC031091D3032091D403021739F0112742
:104630001093D5030093D403102F09C02091D50304
:10464000222329F4002312F0139513951A95109341
:10465000D30320912802121719F02195121729F47B
:1046600011271093D3030093CE030091CF030023AF
:1046700069F511271093CF030091CD0300FF26C0E9
:104680001093CD031091D0032091D103021739F07C
:1046900011271093D2030093D103102F09C020914A
:1046A000D203222329F4002312F0139513951A95AF
:1046B0001093D00320912802121719F02195121798
:1046C00029F411271093D0030093CF030091D00158
:1046D000002309F09DC106E010912702112329F45F
:1046E0000091370106FD1FC00BE00093D5010027A4
:1046F0000093D1010093D6010FEF0093D0010091F8
:10470000CC01002371F0023061F000E200937903E4
:1047100000937A0300937B0300937C0300E20093F1
:10472000AB020C948C1300919901002309F078C01E
:1047300000913A0104FD2DC00FEF00939901F89408
:1047400000913401037F00933401009335010095FB
:1047500000933A0110E60E944E33009132010F7728
:10476000009332010093330100950093370110E369
:104770000E944E330FEF0093C9030093CA03002732
:104780000093CB010091C804077F0093C8040C94E8
:104790008C1300919A01002309F008C000913A019E
:1047A00000FD24C30FEF00939A019EC40AE000931A
:1047B00028024091CF0340FF24C010E00E941F3424
:1047C000102F0E70069547FF04C00A9532F407E0DB
:1047D00004C0039508300CF00027000F00930D046F
:1047E0002091C80423FF00930E04117F012B0E9328
:1047F000F89400270093CF030FEF009327027894DB
:1048000073C400913A0100FF6FC4002700939A011E
:104810000093D0030093D20301E000932802E6C284
:104820000AE0009328020091C903002341F000919F
:10483000C801002321F40093C9030E94463400916B
:10484000CA03002341F00091C601002321F4009324
:10485000CA030E9461341091CE0310FD1BC0F8946E
:1048600000913A0102FD0AC00091A902002311F053
:104870000C948C130FEF0093A90221C003FD4BC0D1
:104880000091AA02002311F00C948C130FEF0093F7
:10489000AA0206C0F89429E01091CE0317FF0FC0BA
:1048A0000091AA040A9500230AF401E30093AA04E4
:1048B0000E94303417FD12C02A9591F72CC0009148
:1048C000AA040395023309F400270093AA040E9466
:1048D000303417FD03C02A9591F71DC010E00E94E7
:1048E0001F340E7000930D041091C80413FF009341
:1048F0000E040E9406340FEF009327020093C603B4
:104900000093DE03002700935402009355020093A6
:10491000CE030C948C134091CF0340FF5FC047FF40
:104920001DC00091AA040023A1F0053091F00A30C7
:1049300081F00F3071F0043161F0093151F00E3126
:1049400041F0033231F0083221F00D3211F00A95B6
:104950001CC000270093CF030C948C130091AA0471
:104960000430B9F30930A9F30E3099F3033189F318
:10497000083179F30D3169F3023259F3073249F303
:104980000C3239F3013329F303950F930E9430342D
:104990001F771C930F910093AA040E943034106873
:1049A0001C9310E00E941F340E7000930D041091B0
:1049B000C80413FF00930E040E9406340FEF009307
:1049C000C6030093DE0300932702002700935402DE
:1049D000009355020093CF030C948C131127009180
:1049E0003A0104FF0EC01093990100270093D303EE
:1049F0000093D0030093D5030093D20301E000930A
:104A0000280200912702002309F44BC40C948C1354
:104A10000091D301002311F00C948C131091D50157
:104A2000112339F11A951093D5010091D6012091E7
:104A3000D101201710E029F420912702222309F444
:104A40001FEF2091CF010E949E2E0091D601039569
:104A500016E020912702222309F41BE0011709F434
:104A600000270093D6019093D4019093D3010C9426
:104A70008C1300912702002349F00027009327029E
:104A80000093D2010093D0010C948C130091370154
:104A900006FDEFC0112700913A0100FF1FEF1093B0
:104AA0009A01112331F10091CF0300FF0C94792575
:104AB0001127109359021093EC031093ED031093F8
:104AC000D6011091CF01139507FD125022F011313C
:104AD0001CF0112701C010E11093CF0100270093B3
:104AE000CF0306E00093D1010BE00093D5010C94B5
:104AF0008C130AE010915902112321F00BE000936E
:104B0000D5010AE0009328022091CE0320FF2AC09D
:104B100000270093CE0300919A01002331F0002773
:104B200000939A010FEF00939B010091D10127FDA3
:104B30000A9507FD0AE00093D6010091D101200FEC
:104B40000AE022F02B3000E009F0022F0093D1019F
:104B500002E00093D50100270093EC030093ED03DE
:104B60000C948C130091CF0300FF0C948C13F7E18D
:104B7000E6E21091CF0125E0129F22271091D1018A
:104B80001630DCF1100D4091CF014D3069F04E3000
:104B900059F0193291F540910404442309F05DC0A5
:104BA0004FEF4093020429C04091ED03040F43E509
:104BB00022F04427043509F0402F4093ED031FEF06
:104BC0001093E9031091D10116500091CF010D50BF
:104BD00025E0029F100D1F7012952227B7E0A9E46F
:104BE000A10FB21F0091EC03A00FB21FF6E0E6EC9C
:104BF000E40FF20F04910C9330C0110F221F110F1C
:104C0000221FE10FF21F15914591742F5591649168
:104C10000E940D34802F4A9512F00695FCCF20910A
:104C2000CF03052321F0061741F0020F09C022230C
:104C30003AF0662329F0020F03C022230AF4020F80
:104C40007A951AF0000F550FFBCF50958523082B4E
:104C5000F8940C930E940634789411271093CF0394
:104C600001E00093D5010091D1010093D6010C948D
:104C70007F2900270093590210919A01112329F0EE
:104C800000939A010FEF00939B010091D101002343
:104C900062F001E00093D5010091D1010093D601AB
:104CA0000FEF0093D1010C948C130091D2010023DB
:104CB000A9F40FEF0093D2010091E9030093EA03F6
:104CC000F5E0ECEAB1E0A7ED0EE00E9401340EE061
:104CD0000093D4010093D3010C948C130091DF0452
:104CE00015E0019F800123E033270E948743009352
:104CF0000A041093090400270093D2010093D00105
:104D00000093EC030093ED030093D3030093D003CF
:104D10000093D5030093D2030093E90301E00093CD
:104D200028020091D30400FF0FC00E7F0093D3042C
:104D3000002700939E0618E7B4E0A4E10D931A95AE
:104D4000E9F70FE700939D0610E00E941F340E70F4
:104D500000930D04102F0091C80403FD1091AB04C3
:104D60001E7010930E040FEF009327020093DE03D2
:104D7000009351030093640200938B020091CC01D5
:104D8000002399F0023089F00DE40093790300913B
:104D9000E60300937A030091E70300937B030AE3A1
:104DA00000937C0300E20093AB020091DA040C70E4
:104DB0001091F103011711F40C948C130093F1037B
:104DC000BB27AA27002351F0BDEDA0ED043031F040
:104DD000BBEBA0EA003111F0B7E7A0E4F894B09380
:104DE000F203A093F30378940C948C130091C80100
:104DF000002309F08EC00091CB0100FF23C00023E7
:104E00007AF400270093CB01F8940091C804077F3F
:104E10000093C80478940E9446340E94613479C09B
:104E200000270093CB01F8940091C8040860009318
:104E3000C80478940091AB040E7000930E040E9495
:104E40007C3467C0F8940091C70110913A017894BE
:104E500000FF03C00023C2F452C00091AA02002345
:104E600009F057C013FD55C00091C804087009F43B
:104E700050C01FEF1093AA020E9405430E947C3489
:104E80000FEF0093270245C00091B704006800931C
:104E9000B70402E50093A7010AE30093A80120915B
:104EA0004E012093A90110914F011093AA01009186
:104EB00050010093AB01009151010093AC010091AE
:104EC00052010093AD01009159010093AE01009190
:104ED0005A010093AF0100915B010093B001009172
:104EE000DB04002341F00E9413442093A801109397
:104EF000A9010093AA0105E10093C80107C00E941F
:104F000046340091B7040F770093B704002700934D
:104F1000C7011091C8040091C601002339F0187030
:104F200009F439C000270093CA01C4C0187009F4FD
:104F300021C00091A902002309F0BCC00027009302
:104F4000CA0100913A0102FDB5C01FEF1093A902FA
:104F500010E00E941F34F8940093AB040D9100936D
:104F6000AC040D910093AD040D910093AE040E942A
:104F70007C34A0C01091B7040091C901002359F0FE
:104F800012F0116003C00E9461341E7F1093B704B9
:104F900000270093C90100270093CA0140913A01FC
:104FA00043FD41C04FEF4093CA014091370147FD97
:104FB00020C00091A802002309F01BC00FEF00934E
:104FC000A802F8940091AF041091B004012B109145
:104FD000B104012B1091B204012B59F0002700936A
:104FE000AF040093B0040093B1040093B2040E9494
:104FF00006340091CF0300FF16C0F8943091AF043F
:105000002091B0041091B1040091B2040E94532E7B
:105010003093AF042093B0041093B1040093B20412
:105020000E940634789440913A0142FD5DC04FEFF2
:105030004093CA014091370147FD21C00091A80269
:10504000002309F01CC00FEF0093A802F894009110
:10505000B3041091B404012B1091B504012B1091ED
:10506000B604012B61F000270093B3040093B4044D
:105070000093B5040093B6040E940634789400911E
:10508000CF0300FF31C0F8943091B3042091B404F1
:105090001091B5040091B6040E94532E0093B604FB
:1050A0001093B5042093B4043093B3040E940634E3
:1050B00078941AC00091CF0300FF16C0F89411E055
:1050C0000E941F340170302F2D911D910C910E9470
:1050D000532E0C931E932E930E910E7F3170302B16
:1050E0003C930E940634789410E00E941F34302FC5
:1050F00031702D911D910D914091C804487009F0B7
:1051000039C04091AC02442309F034C04091CA0137
:10511000442309F02FC04091CF0340FF2BC0F894E7
:105120000E94722E789488277727662754E640914C
:10513000D804442309F05AE040913A0141FD08C0E7
:1051400067E250E14091D804442311F063E058EE47
:105150004091CF03442352F441E0509560957FEF96
:105160008FEF540F40E0641F741F841F050F161F3C
:10517000271F381F44274093CF034091AC0244239C
:1051800009F08FC09091CE0390FD25C04091E503BA
:1051900040FD0BC047FD19C04091360142FD0CC0D7
:1051A000F89444604093360178949091E5039E7F93
:1051B0009093E50391E00FC043FF02C00C941B29BC
:1051C000F89448604093360178944091E5034F7716
:1051D0004093E5039FEF44274093CE03F8940E9449
:1051E000722E8827772766275AE04091D8044423F7
:1051F00009F051E040913601427029F040913A01A6
:10520000789441FD08C063E058EE4091D8044423EF
:1052100011F0662754E6992352F441E050956095C9
:105220007FEF8FEF540F40E0641F741F841F050F42
:10523000161F271F381F70E067E051EA4FE1401B3F
:10524000510B620B730B6AF571E069EC53EC40E8AB
:10525000401B510B620B730B22F13F932F931F9353
:105260000F9310E00E941F34302F31702D911D914B
:105270000D914F915F916F917F91041739F415173C
:1052800029F4261719F4371709F40BC0F8944E9334
:105290005E936E930E910E7F702B7C930E9406346A
:1052A000789410E00E941F34302F31702D911D91A1
:1052B0000D914091C804487051F540913A0143FD69
:1052C00026C07091AF046091B0045091B104409138
:1052D000B204040F151F261F371F70E067E051EA64
:1052E0004FE1401B510B620B730B4AF471E069EC08
:1052F00053EC40E8401B510B620B730B42F410E07F
:105300000E941F34302F31702D911D910D918827EF
:1053100071E06BEA5EE34FEF401B510B620B730BC6
:105320000AF08FEF809304040F931F932F933F9302
:10533000552745E00E94AF2D0091EF03002329F08F
:1053400000910408002309F47AC00091C5010023EC
:1053500009F075C0E2EBF1E0AEE4B1E089E0772757
:105360000091B803002341F00091340106FD67C0AD
:1053700000270093B80375E10C911191011759F0C2
:10538000813039F4003229F40091D804002309F463
:1053900002C01C9375E111968A9521F0843061F763
:1053A0001696EACF0091D804002319F410E2109366
:1053B0005C01209102041127772319F4222309F4B8
:1053C0003EC01093020475E10091DB04002309F450
:1053D00034C07BE1222311F077E21FEF1093030426
:1053E00020914E0110914F017F930E9413447F91B1
:1053F00020936F011093700100937101009150018F
:1054000000937D010091510100937E0100915201B2
:1054100000937F0100915A010093810100915B018B
:105420000093820100915C01009383010091D804F4
:10543000002319F400E2009383017093C5013F91AA
:105440002F911F910F9174E063E35EE048ED80912E
:10545000B804882321F474E06CE25DE140E88091B7
:105460000D04883011F18A3001F174E063E356E1F4
:1054700048EA8091B804882321F474E06CE25AE38E
:105480004CEC80910D04803081F0843071F08C30D0
:1054900061F074E063E357E048E08091B80488234A
:1054A00021F474E06CE250E044E37F936F935F93E8
:1054B0004F93040F151F261F371F00931C081093CE
:1054C0001D0820931E0830931F0840914D025AE09A
:1054D000459FECE7F0E0E00DF11D772765915591D0
:1054E0004591332722271127002780910D0488300A
:1054F000A1F08A3091F015910491843071F08C30D4
:1055000061F0803051F0009510952095309581E044
:10551000080F80E0181F281F381F400F511F621FFF
:10552000731F0F911F912F913F914F935F936F9333
:105530007F93041B150B260B370B7091D6036091DC
:10554000D7035091D8034091D903041B150B260BA8
:10555000370B0093200810932108209322083093E2
:10556000230840914E025AE0459FECE1F2E0E00D45
:10557000F11D3327259115910591772766275591C0
:10558000449180910D04843069F08C3059F0803062
:1055900049F0863089F08E3079F0823069F05527F5
:1055A00044270AC081E07095609550954095480F5A
:1055B00080E0581F681F781F040F151F261F371F14
:1055C0007F916F915F914F91040F151F261F371F19
:1055D0007091D6036091D7035091D8034091D903BD
:1055E000040F151F261F371F7091DA036091DB032C
:1055F0005091DC034091DD03041B150B260B370B88
:105600000093240810932508209326083093270838
:1056100040914E025AE0459FECE1F2E0E00DF11DB1
:105620003327259115910591772766275591449148
:1056300080910D04883049F08A3039F0803051F083
:10564000843041F08C3031F00FC000271127222721
:10565000332730C081E07095609550954095480F94
:1056600080E0581F681F781F040F151F261F371F63
:1056700077276627509117014091180180910D04FA
:10568000823041F0803051F481E070956095509502
:105690004095480F040F151F261F371F7091DA031E
:1056A0006091DB035091DC034091DD03041B150B7B
:1056B000260B370B009328081093290820932A08FB
:1056C00030932B0880910E044DE730E023EA1FED64
:1056D00003EB883029F14091DD0430E023EA13ED3B
:1056E0000BEF8630E9F08E30D9F04DE730E023EA59
:1056F0001DE300E18A30A1F0803091F0823081F02A
:105700004091DE0430E023EA1DED0BE55091DA0410
:1057100057FF06C04091DE0430E023EA0BE61BEEA3
:105720005527440F551F440F551F440F551F440F55
:10573000551F6627040F151F261F361F00932C08C0
:1057400010932D0820932E0830932F080E943C348C
:105750003E91317011962D911D910D914091340122
:1057600044FD14C04091C804487081F440913A014E
:1057700042FD0CC07091B3046091B4045091B50423
:105780004091B604040F151F261F371F0F931F9358
:105790002F933F938091340186FD04C08091DA04F9
:1057A000807161F470912F0860912E0850912D083E
:1057B00040912C08040F151F261F371F0093300837
:1057C000109331082093320830933308882771E012
:1057D0006FE451EB40E80E94F4330AF0826080935A
:1057E00099028091DA04807109F056C03F912F919F
:1057F0001F910F910F931F932F933F93882771E071
:105800006BEA5EE34FEF401B510B620B730B0AF028
:105810008FEF90910404892B809304040E949F438E
:10582000A6F000910E040430BCF10A30A9F10091F9
:10583000340106FD31C00027009330080093310881
:10584000009332080093330827C01091DA0415FD45
:1058500011C00027009330080093310800933208EC
:105860000093330800932C0800932D0800932E0812
:1058700000932F080091B803002371F400913401C4
:1058800006FF0AC00091B703002331F407E100933B
:10589000B7030FEF0093B803442736E0ACE1B8E05C
:1058A000C4E3D8E024E00D911991011709F041609B
:1058B0002A95C9F7440F3A95A9F7442309F48CC0F7
:1058C000F8944F9346FF13C000911C0800933408CE
:1058D00010911D081093350820911E08209336085A
:1058E00030911F083093370848E20E94692D4F918C
:1058F0004F9345FF13C00091200800933808109182
:105900002108109339082091220820933A083091F9
:10591000230830933B0840E20E94692D4F914F933A
:1059200044FF13C00091240800933C0810912508FF
:1059300010933D082091260820933E0830912708B7
:1059400030933F0848E10E94322D4F914F9343FF1F
:1059500013C0009128080093400810912908109363
:10596000410820912A082093420830912B08309357
:10597000430840E30E94322D4F914F9342FF13C0E2
:1059800000912C080093440810912D0810934508AD
:1059900020912E082093460830912F083093470815
:1059A00040E10E94322D4F9141FF13C00091300819
:1059B000009348081091310810934908209132084B
:1059C00020934A083091330830934B0848E30E94F3
:1059D000322D0E94AB2D78943F912F911F910F9102
:1059E000409199014423E1F540919A014423C1F586
:1059F0004091C804487021F440913A0142FD30C002
:105A0000552745E00E94AF2D0091C601002341F5C6
:105A1000E2EBF1E0A1E9B1E088E077270C91119188
:105A2000011711F01C9375E111968A9509F0F6CFD4
:105A30007093C60108E500938F010AE3009390017B
:105A40000091DB04002361F02091910110919201FB
:105A50000E941344209390011093910100939201AE
:105A60000C948C134F93332352F40095109520958A
:105A7000309541E0040F40E0141F241F341F67E1FC
:105A80005BED41E970910A04470F70910904571FBB
:105A900070E0671F0E94A6302F912F9301E00E94B3
:105AA00083330091DF032F912F930E948333009162
:105AB000E0032F912F930E9483330091E1032F91F4
:105AC0002F930E9483330091E2032F910E9483332E
:105AD00008954F93332352F40095109520953095F7
:105AE00041E0040F40E0141F241F341F6EE050E516
:105AF0004AE87091DF04470F70E0571F671F0E944C
:105B0000A6302F912F930091DF0314E00E94CA3337
:105B10000091E0032F912F9315E00E94CA3300916A
:105B2000E1032F912F9316E00E94CA330091E20304
:105B30002F912F9317E00E94CA330091E3032F9116
:105B40002F9318E00E94CA330091E4032F9119E0CB
:105B50000E94CA3308952F9A00002F9808955F93EA
:105B60004F9340E233235AF43095209510950095D9
:105B700041E0040F40E0141F241F341F4DE24F93F7
:105B800044275527662778E183E090E3000F111F33
:105B9000221F331F441F551F661F7A9589F160939A
:105BA0002F01680F63FF60912F0160932F01690F30
:105BB00067FF60912F0150932F01580F53FF5091B1
:105BC0002F0150932F01590F57FF50912F014093F0
:105BD0002F01480F43FF40912F0140932F01490FA0
:105BE00047FF40912F0130932F01380F33FF309141
:105BF0002F0130932F01390F37FF30912F01C6CF7E
:105C00001F910F912EE2A1EBB1E01D93762F7295BB
:105C10007F7070637D93013009F42D936F70606322
:105C20006D93023009F42D93752F72957F70706318
:105C30007D93033009F42D935F7050635D930430BE
:105C400009F42D93742F72957F7070637D930530E6
:105C500009F42D934F7040634D93063009F42D9352
:105C6000732F72957F7070637D93073009F42D93C5
:105C70003F7030633D93083009F42D935F915523B5
:105C800009F00895199721E03D91303349F4021746
:105C900039F0129730E23D931D9323952930A1F7F7
:105CA00012971C9308954091AC02442309F0089583
:105CB0000E94722E7727662755274AE080913A0185
:105CC00081FD02C053E048EE8091CF0388232AF47F
:105CD000041B150B260B370B0895040F151F261FE9
:105CE000371F08950F9300913A0101FD25C00091DF
:105CF000DA04037059F00130B1F0023069F005E7C1
:105D000000939B0600E300939C0613C000270093BA
:105D10009B0600939C060DC00AE300939B0608E9CE
:105D200000939C0606C003E100939B0608E80093DD
:105D30009C0600270093AC020F910895422FE0EBE0
:105D4000F5E1442309F440C0E6ECF5E14130E1F12E
:105D5000ECEDF5E14230C1F1E2EFF5E14330A1F1C4
:105D6000E8E0F6E1443081F1EEE1F6E1453061F141
:105D7000E4E3F6E1463041F1EAE4F6E1473021F1AF
:105D8000E0E6F6E1483001F1E6E7F6E14930E1F01E
:105D9000ECE8F6E14A30C1F0E2EAF6E14B30A1F07E
:105DA000E8EBF6E14C3081F0EEECF6E14D3061F0DD
:105DB000E4EEF6E14E3041F0EAEFF6E14F3021F04B
:105DC000E0E1F7E1403101F0043039F42091C904F9
:105DD000287019F0F5E1E4EA0DC0000F2227E00F6A
:105DE000F21F069535912491330F221FF8E0EAED5A
:105DF000E30FF21FD1E0C7ED26E0922F35913993E2
:105E00002A95E1F72FE1299328E2299327E62993A0
:105E100021E0299329939B5F112339F02FE12993E6
:105E200022E7299321E029939D5F2591222349F4BC
:105E30003591309326012591299393953A95D9F779
:105E40002591043029F43091C904387009F0B6C0A6
:105E5000B7E1A6E235E0439F06300CF0000D442781
:105E6000000F441F000F441FA00FB41F35913323B0
:105E7000EAF1FF93EF93FD014491EF91FF914034DC
:105E8000ACF04A349CF440544F704295B7E0A9E41A
:105E9000A40F40E0B41F3CE02D91222329F0299368
:105EA00093953A95C9F78AC020E284C0442740936D
:105EB000CB031F93FF93EF93FD01159145915591EE
:105EC00064910E940D344A9512F00695FCCF05238B
:105ED000039FEF91FF911F91E00DF11D259122236A
:105EE00021F0299393953A95C9F768C04FEF55274C
:105EF000222312F444275FEF409359025093CB03BF
:105F00003195432F1F939F93CF93DF93FD01BB27C1
:105F1000A491552339F01A2F0E940D3433272227DC
:105F2000112705C0B1E0332722271D910C91552779
:105F30000E94AF2DDF91CF919F911F91009126017B
:105F400031E1301B313079F1323041F1333009F138
:105F50003430D1F0353099F0363061F0373029F0F7
:105F60000091B201099393953A950091B301099379
:105F700093953A950091B401099393953A950091C0
:105F8000B501099393953A950091B60109939395BC
:105F90003A950091B701099393953A950091B8010C
:105FA000099393953A950091B901099393953A9580
:105FB00029F020E2299393953A95E1F7112339F0DE
:105FC0000FE1099302E7099300E009939D5F0895AB
:105FD000F8943091310130653BB93FEF37B93091DA
:105FE000390138B9439A449829980E9494300E9404
:105FF0009430299A0E949430449A29980E949430AF
:106000000E949430299A0E9494300E9494304398C0
:1060100029980E9494300E949430299A0E949430CA
:106020000E9494300E3961F40E944730012F0E9483
:106030004730022F0E94473000270E94473008C097
:106040000E944730012F0E944730022F0E944730A4
:106050000E9494300E949430449A29980E9494306F
:106060000E949430299A0E949430439A29980E9461
:1060700094300E949430299A0E9494304498299830
:106080000E9494300E949430299A7894089538E0C0
:10609000449A000F08F4449829980E9494300E9472
:1060A0009430299A439A29980E9494300E949430FF
:1060B000299A0E949430439829980E9494300E9413
:1060C0009430299A0E9494300E9494303A9501F7B6
:1060D000449829980E9494300E949430599A439A87
:1060E00029980E9494300E949430299AC0913101DD
:1060F000C062CBB9CC27C7B929980E9494300E94BE
:106100009430C6B1299AC0913101C065CBB9CFEFA7
:10611000C7B9C0913901C8B9439829980E949430F1
:106120000E949430299A0895000000000895F9997A
:10613000FECFB2BDA1BDF89A00B50895F999FECF82
:10614000B2BDA1BD00BDFA9AF99A08957727709360
:10615000DF037093E0037093E1037093E2037093A5
:10616000E3037093E40340FD0E94BD3066955795AC
:10617000479573957631B9F7089588279927A32F06
:10618000B22FC12FD02FE72FEE2341F0DD0FCC1F10
:10619000BB1FAA1F991F881FEA95F6CFE091E40361
:1061A000DE0FD093E403E091E303CE1FC093E3033B
:1061B000E091E203BE1FB093E203E091E103AE1F62
:1061C000A093E103E091E0039E1F9093E003E09130
:1061D000DF038E1F8093DF0308950091C8040078C9
:1061E00041F5002700930108009347010093C50182
:1061F0000093C8010093C6010093D3010093C1022C
:106200000093C20200938E030093AB0200938F03AE
:106210000093B7030093C5030093C7030093500393
:10622000009308040093120400935C0200935D0243
:10623000089501E010904501011509F488C1039506
:10624000011509F4F8C10395011509F4C3C00395BC
:10625000011509F4DCC00395011509F4E6C00395A6
:10626000011509F4F0C00395011509F4FCC003956C
:10627000011509F406C10395011509F410C1039530
:10628000011509F41AC10395011509F424C10395F8
:10629000011509F42EC10395011509F438C10395C0
:1062A000011509F442C10395011509F4AFC1039525
:1062B000011509F45AC10395011509F491C103951B
:1062C000011509F460C10395011509F47AC101E0D3
:1062D00020900108222009F03AC10091EF03002329
:1062E00061F000910408002309F4B4C10091020890
:1062F00010910308012B09F0ADC102E02090470185
:10630000222009F098C103952090C501222009F0B0
:1063100061C003952090C801222009F078C0039540
:106320002090C601222009F080C003952090D3015F
:10633000222009F088C003952090C102222009F094
:1063400092C003952090C202222009F09AC00395C2
:1063500020908E03222009F0A2C003952090AB026A
:10636000222009F0AAC0039520908F03222009F073
:10637000B2C003952090B703222009F0BAC003955C
:106380002090C503222009F0C2C00395209050033D
:10639000222009F0CAC003952090C703222009F0EB
:1063A00035C1039520900804222009F0DEC0039532
:1063B00020901204222009F013C1039520905C0262
:1063C000222009F0E0C0039520905D02222009F010
:1063D000F8C040C10093450104E1E8E4F1E0109108
:1063E000DB04112359F0E9E6F1E00AE1109103041E
:1063F000112321F01CE0010FE11BF0402090C501AA
:106400002A942092C5010219102E442427C100931A
:1064100045012090C8012A942092C80104E1021984
:10642000102EECE9F1E0442419C1009345012090BD
:10643000C6012A942092C60104E10219102EE4E854
:10644000F1E044240BC1009345012090D3012A942C
:106450002092D3010091D4010A950219102EE7ED84
:10646000F1E04424FBC0009345012090C1022A942E
:106470002092C10200E10219102EE0EBF2E0442468
:10648000EDC0009345012090C2022A942092C202DE
:106490000FE60219102EE4ECF2E04424DFC0009372
:1064A000450120908E032A9420928E0305E1021963
:1064B000102EE3E5F3E04424D1C000934501209081
:1064C000AB022A942092AB020FE10219102EEEE6E5
:1064D000F3E04424C3C00093450120908F032A9425
:1064E00020928F030EE00219102EE1E9F3E044241C
:1064F000B5C0009345012090B7032A942092B703BA
:1065000006E10219102EE0EAF3E04424A7C000934C
:1065100045012090C5032A942092C5030BE002197F
:10652000102EE9EBF3E0442499C01091370116FFD7
:1065300091C000934501209050032A94209250036B
:106540000BE10219102EE4E3F3E0442487C000932A
:106550004501209001082A942092010807E10219C0
:10656000102EE9EEF7E0442479C000934501209015
:1065700008042A942092080406E10219102EE5E08E
:10658000F8E044246BC000934501112720905C0281
:1065900027FE02C021941FEF2A9420925C0209E199
:1065A0000219102E043144F0112331F01394139486
:1065B0001394139413941394EEE7F6E04424409458
:1065C0004DC00093450120905D022A9420925D0207
:1065D0000BE10219102EEEE9F6E0442440943EC08F
:1065E00000934501209012042A94209212040BE09B
:1065F0000219102E0B3029F40091110405FD01C081
:106600001394E4E2F6E04424409428C0009345014A
:106610002090C7032A942092C70304E00219102E89
:10662000E2E5F5E00091C803002311F4ECE4F5E0A5
:106630004424409413C000934501209047012A94BC
:106640002092470103E10219102EE8E3F5E044240B
:10665000409404C0222420925A0208950AE0009334
:106660005B0200914501222009F4002700934501B7
:106670002224E10DF21D008040FCC895002D1FEF83
:1066800017B918B90E9494300E94943008B90E943A
:1066900094302E980E9494302E9A0895F8942FEFFB
:1066A000103328F42FEF28B9222727B904C028B9BE
:1066B00027B9000008B900913101012B0BB9000086
:1066C0000000000029980E9494300E94943006B186
:1066D000299A08950F931F93F894009138010F772A
:1066E0000093380110E40E944E331F910F910E94D5
:1066F0004E330091380100680093380110E40E9485
:106700004E33789408950F932F93F89400913801A5
:10671000022B10E40E944E332F910F9108B90E9472
:1067200094300E949430289A0E9494300E949430B1
:1067300028980E9494300E949430089508B90E94CD
:1067400094300E949430289AAA27B2E0129711F050
:106750001B99FCCF2898AA27B2E0129711F01B9B37
:10676000FCCF0E9494300E9494300895289AAA2762
:10677000B2E0129711F01B99FCCF06B12898AA2716
:10678000B2E0129711F01B9BFCCF0E9494300E9444
:10679000943008950F931F932F93F894009138012C
:1067A000022B10E40E944E332F911F910F91009500
:1067B00008B91F9310952C9814FD2C9A2D9815FD4F
:1067C0002D9A1F9112951095107F00913101012B88
:1067D0000BB90E9494300E949430289A0E94943001
:1067E0000E94943028980895002E041B002D012E3D
:1067F000150B102D022E260B202D032E370B302DBE
:10680000089515911D930A95E1F7089503E100930A
:10681000990608E800939A060895B4E0AAEA1123BD
:106820004AF4B4E0A7EE2091AA0406E0029FA00D6E
:10683000B11D1095A10F10E0B11F0C910895112307
:1068400029F0B4E0AAEA012E112406C0B4E0A7EEB4
:106850001091AA0406E0019FA00DB11D0D910895AD
:10686000B4E0A7EE0091AA0416E0109FA00DB11DA0
:1068700014960D911C91089510E00091C8040870C1
:1068800009F011E00E941F340E70089500E2009399
:10689000A7010093A8010093A9010093AA01009306
:1068A000AB010093AC010093AD010093AE010093E6
:1068B000AF010093B001F89405E10093C80178940A
:1068C000089500E200938F010093900100939101DD
:1068D000009392010093930100939401009395011A
:1068E000009396010093970100939801F89405E1B5
:1068F0000093C60178940895E8ECF5E00091AB04AC
:106900000695077018E0109FE00DF11D05910093AA
:10691000A70105910093A80105910093A901059194
:106920000093AA0105910093AB0105910093AC017E
:1069300005910093AD0105910093AE0100E2009333
:10694000AF010093B00105E10093C8010895B1E0E3
:10695000A2EE0091CB04102F0F7705351CF01078B4
:106960001093CB0416E0019FA00DB11D0E9497303B
:10697000302F317000938B0611960E949730202F94
:1069800020938C0611960E949730102F10938D063D
:1069900011960E94973000938E060F9311960E94D5
:1069A000973000938F0611960E94973000939006BF
:1069B0000F91089545E00E94AF2D0091AB02002396
:1069C00009F008950DE4009379030AE300937C0332
:1069D0000091B20100937D030091B30100937E0307
:1069E0000091B40100937F030091B50100938003EF
:1069F0000091B601009381030091B70100938203D7
:106A00000091B801009383030091B90100938403BE
:106A100000E20093850348E03327222711270091E5
:106A2000CB040E94AF2D0091B80100937A0300932C
:106A3000E6030091B90100937B030093E703E8ECC0
:106A4000F5E000918B060E70069518E0109FE00DA2
:106A5000F11D05910093860305910093870305912D
:106A600000938803059100938903059100938A039D
:106A7000059100938B03059100938C03059100937E
:106A80008D0300E20093AB0208950091A506002358
:106A900009F408950091F706002309F00895F7E03E
:106AA000EEE3B6E0A7EA27E61D911F7D05910117E9
:106AB000C1F40093F9061C911F7D04910117A9F4FC
:106AC0000093FA06119611270C910B3309F41FEF6E
:106AD00010935F023196C591D491FE01D6E0CBEFC1
:106AE000099433962A9511F704C0119733962A9585
:106AF000D9F6D6E0C9EF0FE309930FEF00935F02D9
:106B000002E011C03327222711275FEF48E00E94DF
:106B1000AF2D0091B70109930091B801099300913D
:106B2000B901099306E01BE318830093F80600936C
:106B3000F7060091C10000620093C1000027009396
:106B4000A50600915F0200FF0E94063408951123FC
:106B500071F010E30091320105FD11E319931993CF
:106B600010E30091110407FD11E319931AC00D9170
:106B700009930E94A24202300AF0BBCF302F0E943C
:106B8000A24202300AF0B5CF10913201332329F42A
:106B900015FD1F7D1093330104C015FF1062109383
:106BA000330106E0C0CF112341F000916B02409108
:106BB0006D0240FD00916C02A5CF63E00E946B4224
:106BC0000AF497CF222309F094CF10936C020FEFB1
:106BD00000936D0206E0A7CF112341F000916F02F0
:106BE0004091710240FD009170028CCF63E00E94E1
:106BF0006B420AF47ECF222309F07BCF1093700200
:106C00000FEF0093710206E08ECF112349F010E3DD
:106C10000091DA04007409F011E3199304E083CFC2
:106C20000E94A24202300AF064CFF8941091DA0474
:106C30001F7B012B0093DA04789404E074CF1123B6
:106C400069F00E943C3413960C91087006950695E5
:106C500006950395005D099304E065CF0E94A2426A
:106C6000013019F0023009F044CF0A95000F000FEF
:106C7000000F0F93F8940E943C3413960C91077FF9
:106C80001F91012B0C9378940FEF0093270204E0DF
:106C90004ACF112361F00E943034007106950695A9
:106CA000069506950395005D099304E03CCF0E948C
:106CB000A242013019F0023009F01BCF0A95000FF3
:106CC000000F000F000F0F93F8940E9430340E91C4
:106CD0000F7E1F91012B0C9378940FEF00932702E6
:106CE00004E021CF112349F010E30091C8040170A2
:106CF00009F011E3199304E016CF0E94A24202307A
:106D00000AF0F7CEF8941091C8041E7F012B00936F
:106D1000C804789404E007CF112349F010E30091F0
:106D20003B01007809F011E3199304E0FCCE0E94C6
:106D3000A24202300AF0DDCEF8940F930E94303464
:106D40000F7D1F91110F110F110F110F110F012B3B
:106D50000E93789404E0E7CE112339F00091D1042A
:106D600010E3010F099304E0DECE0E94A242083036
:106D70000AF0BFCEF8940093D104789404E0D3CE07
:106D8000112319F00091DC04BDCE63E00E946B4238
:106D90000AF4AFCE222309F0ACCE1093DC0406E057
:106DA000C2CE112349F010E30091DA04007109F01A
:106DB00011E3199304E0B7CE0E94A24202300AF018
:106DC00098CEF8941091DA041F7E002311F000E1B0
:106DD000102B1093DA04789404E0A5CE0027112339
:106DE000A9F00091D6048ECE01E0112379F0009134
:106DF000D60488CE02E0112349F00091D60482CE59
:106E000003E0112319F00091D7047CCE0F9363E0C7
:106E10000E946B420F910AF46CCE222309F069CED6
:106E2000202F06E0222319F41093D6047CCE2130C3
:106E300019F41093D60477CE223019F41093D604A7
:106E400072CE1093D7046FCE112319F00091DE0497
:106E500059CE63E00E946B420AF44BCE222309F024
:106E600048CE1093DE0406E05ECE112319F00091A7
:106E7000DD0448CE63E00E946B420AF43ACE22233E
:106E800009F037CE1093DD0406E04DCE112319F042
:106E90000091D50437CE63E00E946B420AF429CEFC
:106EA000222309F026CE1093D50406E03CCE112310
:106EB00049F010E30091DA04007209F011E319932C
:106EC00004E031CE0E94A24202300AF012CEF894C1
:106ED0001091DA041F7D002309F010621093DA0488
:106EE000789404E020CE112319F00091DF040ACE3B
:106EF00063E00E946B420AF4FCCD222309F0F9CD35
:106F00001093DF0406E00FCE0091E50300680093C4
:106F1000E50303E008CE112319F00091C604F2CD79
:106F200063E00E946B420AF4E4CD222309F0E1CD34
:106F30001093C60406E0F7CD112349F010E3009149
:106F4000D904007409F011E3199304E0ECCD0E9418
:106F5000A24202300AF0CDCDF8941127002309F0A7
:106F600010E41093D904789404E0DDCD112339F0B6
:106F700010E30091E004010F099304E0D4CD0E94D6
:106F8000A24203300AF0B5CDF8940093E00478945F
:106F900004E0C9CD112349F010E30091DA04007830
:106FA00009F011E3199304E0BECD0E94A242023021
:106FB0000AF09FCDF8941091DA041F77002309F0AE
:106FC00010681093DA04789404E0ADCD0091E503E5
:106FD00001600093E50303E0A6CD112321F010E04A
:106FE0000E94A642A0CD10E00E94CF420AF481CDBB
:106FF0009ACD112321F011E00E94A64294CD11E018
:107000000E94CF420AF475CD8ECD112349F010E3D2
:107010000091C904087009F011E3199304E083CDCD
:107020000E94A24202300AF064CDF8941091C90483
:10703000177F002309F018601093C904789404E0C6
:1070400072CD112391F00091D2040F7733272227BC
:1070500011275FEF48E00E94AF2D0091B80109931E
:107060000091B901099305E05ECD62E00E946B4298
:107070000AF43FCD222309F03CCD15310AF039CD79
:10708000F8940091D2040078102B1093D2047894D5
:1070900005E049CD112339F00091B80410E3010F48
:1070A000099304E040CD0E94A24202300AF021CDB3
:1070B0000093B80404E037CD112321F024E0F4E07C
:1070C000EDEB0FC00C91005302300AF012CDF4E04A
:1070D000EDEB442734E019C0112379F024E0F4E00B
:1070E000E9EB019110E30A3012F011E60A50010FAA
:1070F00009932A95B1F707E016CD0C91003309F0FA
:10710000F8CCF4E0E9EB4FEF34E00E94A2424423D4
:1071100089F40A308AF0102F10620AE0113361F00E
:107120000395123349F00395133331F0039514336B
:1071300019F0DFCC0930EAF701933A9531F707E00F
:10714000F2CC112321F000E3099304E0ECCC0E947F
:10715000A24210E3002351F0013019F0023021F077
:10716000C8CC0E94054302C00E9431430091C8046C
:10717000077F0093C80404E0D6CC112349F000E354
:107180001091C804187009F001E3099304E0CBCC16
:107190000E94A24210E3002351F0013009F0A9CC73
:1071A0000091C80408600093C80404E0BCCC0091BE
:1071B000C804077F0093C80404E0B5CC112349F04C
:1071C00010E300913A01027009F011E3199304E011
:1071D000AACC0E94A24202300AF08BCCF894109103
:1071E00034011D7F000F00950270012B00933501C3
:1071F000789404E098CC00910B04002309F04AC075
:10720000112321F110E00E941F34007340910D04FE
:1072100044305CF04C304CF410E3199319931993FB
:10722000002309F411E3199374C0003224F031F003
:1072300010E324E305C012E324E302C011E328E3D2
:107240001993299310E31993199363C064E00E9482
:107250006B420AF44ECC40910D0444305CF04C304B
:107260004CF412300CF045CC109511701295212F72
:107270003FEC44C038EE43E01317240700E338F036
:1072800030ED47E01317240700E208F000E1202F5B
:107290003FEC34C01123A9F010E00E941F3410E32A
:1072A00007FD11E3199310E306FD11E3199310E3B1
:1072B00005FD11E3199310E304FD11E3199307E0B1
:1072C00032CC0E94A24202300CF013CC202F220FAD
:1072D0000E94A24202300CF00CCC202B220F0E9404
:1072E000A24202300CF005CC202B220F0E94A242B9
:1072F00002300CF0FECB202B22953FE010E00E94E4
:107300001F340323022B0E930FEF009351030093BE
:10731000DE0307E008CC112369F010E00E941F345F
:10732000007C029506950695039510E3010F0993DD
:1073300004E0F9CB0E94A242002311F005300CF0CA
:10734000D8CB0A95000F000F0295202F10E00E9465
:107350001F340F73022B0E930FEF00935103009312
:10736000DE0304E0E0CB112359F010E00E941F344B
:1073700000730295039510E3010F099304E0D3CB4A
:107380000E94A242002311F005300CF0B2CB0A9506
:107390000295202F10E00E941F340F7C022B0E93C9
:1073A0000FEF009351030093DE0304E0BCCB1123E5
:1073B00059F000E3099309930E9430341076129536
:1073C0001063199306E0AFCB0E94A2420E94A24232
:1073D0000E94A242002339F0023029F0043019F053
:1073E000063009F086CB02950F930E9430341F7946
:1073F0000F91012B0C930FEF0093270206E093CB24
:10740000112349F010E30091E104002309F011E396
:10741000199304E088CB0E94A24202300AF069CBA3
:10742000F8940093E104789404E07DCB07E309939A
:1074300001E3099300E3099306E075CB10E00E9495
:10744000A64200910B040023E1F00091B6041091D4
:10745000B5042091B4043091B3045FEF48E00E947A
:10746000AF2D0091B10109930091B60109930091EC
:10747000B70109930091B80109930091B9010993EB
:1074800006C000E2099309930993099309930091B7
:10749000B2041091B1042091B0043091AF045FEFB9
:1074A00048E00E94AF2D0091B10109930091B6010F
:1074B00009930091B70109930091B80109930091D4
:1074C000B901099310E30091B70407FD11E3199383
:1074D00010E30091B70400FD11E3199310E2199332
:1074E0000091E603006309930091E70300630993A9
:1074F00010E30091340106FD11E319930E944A4400
:10750000199310E30091010400FD12E3199310E3B5
:107510000091000400FD11E3199310E30091C804E9
:1075200003FD11E3199300E309930993099300E222
:10753000099306E2F8CA112341F13091D603209154
:10754000D7031091D8030091D90340910B04442331
:1075500041F03091DA032091DB031091DC030091BC
:10756000DD035FEF48E00E94AF2D0091B101099368
:107570000091B60109930091B70109930091B801F8
:1075800009930091B90109933DC00D91003229F092
:107590000B3219F00D3209F0ACCA09930F9364E075
:1075A0000E946B4212F40F91A4CA012F122F083EC1
:1075B00043E0140718F431E022E30FC0003D47E038
:1075C000140718F432E024E608C0083843E1140731
:1075D00010F00F918ECA33E02AEF306830935602D4
:1075E00033270E9487431F911D3209F401951091A2
:1075F0000B0410FF0093540210FD009355020FEF8F
:107600000093DE0308E08FCA112361F010E30091BC
:10761000C90400730695069506950695010F099312
:1076200004E081CA0E94A24203300AF062CAF894C0
:10763000000F000F000F000F1091C9041F7C102BCA
:107640001093C904789404E06ECA112349F00091A4
:107650001A0110918002112311F000917F0252CA89
:1076600063E00E946B420AF444CA222309F041CA33
:1076700010340AF03ECA15300AF43BCA10937F0258
:107680000FEF0093800206E04ECA112349F010E389
:1076900000913401067009F011E3199304E043CA24
:1076A0000D910993F7E0E9E41CE022270D9109937D
:1076B0000C3309F42FEF01931A95C1F734961CE0AF
:1076C0000D91099301931A95D9F701E0222309F44A
:1076D00000E80093EE030FEF0093EA030CE123CAE6
:1076E000112341F010E30091C9040770010F0993C1
:1076F00004E019CA0E94A24205300AF0FAC9F894BF
:107700001091C904187F102B1093C904789404E0D9
:107710000ACA112339F010E30091AC0200FD11E315
:10772000199310C00E94A2421127002321F01FEFDD
:10773000013009F0DEC91093AC02109510FF1395CB
:107740001093900304E0EFC9112341F010E300917E
:10775000DA040370010F099304E0E5C90E94A24214
:1077600004300AF0C6C9F8941091DA041C7F102B7B
:107770001093DA04789404E0D6C9112349F010E399
:107780000091E404002309F011E3199304E0CBC94C
:107790000E94A24202300AF0ACC9F894889407957E
:1077A00007950093E404789404E0BDC9112351F0D7
:1077B00000E209930091E603006309930091E70357
:1077C000099319C00D9109930D910F930C910F938B
:1077D000119762E00E946B420AF402C015351CF05A
:1077E0000F910F9108C00F910093E7030F91009341
:1077F000E6031093CB0406E096C9112321F00E9402
:107800004A4419932DC00C91099322270333B1F0F8
:107810002395073399F02395023381F023950133A3
:1078200069F02395053351F02395043339F02395FE
:10783000063321F02395093309F05BC9220F10E0CC
:107840000E941F34017F022B0E930E7000930D04D3
:107850001091C80413FF00930E040FEF009327024A
:1078600004E061C9112341F0009172021091750288
:1078700010FD0091740246C963E00E946B420AF455
:1078800038C9222309F035C9109374020FEF009311
:10789000750206E048C90D9109930D91099362E0C4
:1078A0000E946B4215350AF024C9B1E0A2EE06E051
:1078B000019FA00DB11D0E9497300F700F930170B2
:1078C0000F9311960E9497300F9311960E94973054
:1078D0000F9311960E9497301F912F913F915FEF68
:1078E00048E00E94AF2D00E30993099309930091AA
:1078F000B20109930091B30109930091B401099376
:107900000091B50109930091B60109930091B70167
:1079100009930091B80109930091B90109930F915E
:1079200006950E944E44199300E309930993099325
:10793000099300E2099308E1F6C80D9109930D91AE
:10794000099362E00E946B4215350AF0D2C81F937A
:1079500068E00E946B425F910AF4CBC80C9100531F
:107960000AF4C7C80A300AF0C4C809930E946544E3
:10797000660FB1E0A2EE06E0059FA00DB11D042F39
:107980000170062B0E949E301196032F0E949E309C
:107990001196022F0E949E301196012F0E949E3058
:1079A00000E3099309930993099308E1BCC81123E3
:1079B00039F00E94303420E314FD21E3299311C0F3
:1079C0000E94A2423327002321F030E1013009F068
:1079D00090C80E9430341F7E132B1C930FEF00932E
:1079E000270204E0A0C8112341F000916002109129
:1079F000630210FD0091620285C863E00E946B4241
:107A00000AF477C8222309F074C8109362020FEFBA
:107A10000093630206E087C8112371F00E9430349E
:107A20001C70012F10E3002321F011E3043009F052
:107A300012E3199304E077C80E94A24203300AF0CF
:107A400058C8F8940F930E943034137F0F91000FA1
:107A5000000F102B1C93789404E065C8112379F073
:107A600020E3009132010370002320E331F0023063
:107A700021F021E3013009F022E3299318C02C9171
:107A800029933091320130FD3D7F3270203339F03F
:107A900031E0213321F033E0223309F02AC8F89491
:107AA000009133010C7F032B00933301789404E0A1
:107AB0003AC8112301F11127009164022091C804F2
:107AC0002670243031F0263021F033272AE00E943E
:107AD00087433327222711275FEF48E00E94AF2D0D
:107AE0000091B70109930091B80109930091B90180
:107AF000099306E018C863E00E946B4212F40C94EC
:107B000079354091C8044670443051F0463041F018
:107B10001C3010F00C9479350AE0019F102D04C040
:107B2000113810F00C947935109367020FEF009321
:107B3000680206E00C949335112359F010E300918C
:107B4000DA040C7006950695010F099304E00C9475
:107B500093350E94A242043012F00C947935F894C7
:107B60001091DA04137F000F000F102B1093DA042A
:107B7000789404E00C949335112349F000917A0233
:107B800010917D0210FD00917C020C94823563E01F
:107B90000E946B4212F40C947935222311F00C945C
:107BA000793510937C020FEF00937D0206E00C9470
:107BB0009335112351F010E30091D204007809F0BD
:107BC00011E3199304E00C9493350E94A242023011
:107BD00012F00C947935F8941091D2041F77002399
:107BE00009F010681093D204789404E00C94933553
:107BF000112379F010E300910C0420910E0424303D
:107C000024F400FD11E3199314C007FD11E3199347
:107C100010C00E94A242023012F00C947935112754
:107C200000FD10E1009132010F7E012B0093330122
:107C3000789404E00C949335112339F010E300910B
:107C4000F00307FD11E319930DC00E94A242023018
:107C500014F00C947935F89406950795016000931B
:107C6000F003789404E00C949335112331F1332719
:107C70000091820210918302112381F41091170167
:107C800000911801055C104032F400E30993099358
:107C900005E00C94933521E40E94874322271127A5
:107CA0005FEF48E00E94AF2D0091B8010993009169
:107CB000B901099305E00C94933562E00E946B4290
:107CC00012F40C9479351D3010F00C947935109322
:107CD00082020FEF0093830205E00C949335112389
:107CE00051F010E30091C80406700695010F099346
:107CF00004E00C9493350E94A242043012F00C94DC
:107D00007935F8941091C804197F000F102B109347
:107D1000C804789404E00C949335112361F020E3B7
:107D200000913201037019F000FD01C021E310E35E
:107D3000199329931BC00E94A242023014F00C94A4
:107D400079350E94A24232E0013041F000913201C7
:107D500000FD0CC001FF0AC0332700C0F894009159
:107D600033010C7F032B00933301789405E00C94CE
:107D7000933544275527662777271BC07091AF049A
:107D80006091B0045091B1044091B2044A50504007
:107D9000604070400EC07091AF046091B00450918B
:107DA000B1044091B2048AE0480F80E0581F681F78
:107DB000781F7093AF046093B0045093B104409364
:107DC000B20403E00C949335F5E1E3E205910993E5
:107DD00005910993059109930591099305910993DB
:107DE00005910993059109930AE00C9493351123A9
:107DF00049F0009177024091790240FD00917802AC
:107E00000C94823563E00E946B4212F40C94793535
:107E1000222311F00C947935109378020FEF009320
:107E2000790206E00C9493350091E304037011E4A9
:107E3000010F09930EE2099300E309930091E30413
:107E4000069506950395037010E3010F09930EE262
:107E500009930091E30406950695069506950F7023
:107E600010E30A3012F011E30A50199310E3010FE6
:107E700009930AE00C949335112351F100910F04FA
:107E8000099310E0003351F010916903013331F090
:107E900010916D03023311F010916C03012F112723
:107EA00033272CE00E94874322275FEF48E00E949F
:107EB000AF2D0091B60109930091B701099300918C
:107EC000B80109930091B901099308E00C94933526
:107ED0000E94A24212F0043014F00C947935006331
:107EE00000930F0404E00C9493350FEF0093D40437
:107EF00003E00C949335112339F010E30091B7049B
:107F000007FD11E3199318C00E94A24212F002303B
:107F100014F00C9479351091B704002319F417FF6D
:107F200059F002C017FD41F4F8941091340108E0B3
:107F3000102710933501789404E00C949335F8944D
:107F400000913801086010E40E944E3306ED0E9453
:107F50009E3300270E949E33789403E00C9493355F
:107F6000112351F020E30E943034007409F021E322
:107F7000299304E00C9493350E94A242023012F03F
:107F80000C947935F894202F0E9430340F7B2223F3
:107F900009F000640E93789404E00C949335F894FF
:107FA00000913801086010E40E944E3306ED0E94F3
:107FB0009E330FEF10910E041A3019F014300CF0AC
:107FC00000E80E949E33789403E00C9493351123CB
:107FD00039F410E30091000400FD11E318830BC095
:107FE0000E94A242023012F00C947935112700FD54
:107FF0001FEF1093000404E00C949335112341F01B
:1080000010E30091CF04010F099304E00C94933521
:108010000E94A242083012F00C947935F894009333
:10802000CF04789404E00C949335112381F0332726
:10803000222711270091CE045FEF48E00E94AF2D68
:108040000091B80109930091B90109930CC062E055
:108050000E946B4212F40C947935153514F00C948F
:1080600079351093CE0405E00C949335112381F0FB
:108070003327222711270091CD045FEF48E00E94AB
:10808000AF2D0091B80109930091B90109930CC07B
:1080900062E00E946B4212F40C947935153514F0AD
:1080A0000C9479351093CD0405E00C94933511238D
:1080B00041F010E30091D004010F099304E00C9407
:1080C00093350E94A242053012F00C947935F89451
:1080D0000093D004789404E00C949335112341F07C
:1080E00010E30091CC04010F099304E00C94933544
:1080F0000E94A242053012F00C947935F894009356
:10810000CC04789404E00C9493351123C1F0332708
:108110002227009190021AE0019F80015FEF48E062
:108120000E94AF2D0091B60109930091B701099308
:108130000091B80109930091B901099314C064E05A
:108140000E946B4212F40C947935012F122F29E012
:10815000073F120710F00C94793533272AE00E946C
:1081600087430093C50407E00C949335112339F03D
:1081700010E300910B0400FD11E319930BC00E9462
:10818000A242023012F00C947935112700FD1FEF46
:1081900010930B0404E00C94933533272BE11091DA
:1081A000A8040091A9040E94874322275FEF48E0BA
:1081B0000E94AF2D0091B60109930091B701099378
:1081C0000091B80109930091B901099307E00C945B
:1081D0009335112349F0009161024091630240FD03
:1081E000009162020C94823563E00E946B4212F4AB
:1081F0000C947935222311F00C9479351093620296
:108200000FEF0093630206E00C94933510E30091A6
:10821000D30401FD11E319933327222710911B0189
:1082200000911C015FEF48E00E94AF2D0091B60164
:1082300009930091B70109930091B8010993009146
:10824000B901099308E00C9493350E94A2420230D0
:1082500012F00C9479351091D3041B7F000F000F9E
:10826000102B1093D30404E00C949335332722276A
:1082700010911D0100911E015FEF48E00E94AF2D9B
:108280000091B60109930091B70109930091B801DB
:1082900009930091B901099307E00C9493350E946A
:1082A000A242023012F00C9479351091D3041E7F53
:1082B000102B1093D30404E00C949335112321F078
:1082C0000091C7040C94823563E00E946B4212F463
:1082D0000C947935222311F00C9479351093C7044E
:1082E00006E00C949335112321F00091C3040C9403
:1082F000823563E00E946B4212F40C94793522239C
:1083000011F00C947935112311F40C9479351093F4
:10831000C30406E00C9493351123C1F033272227C0
:108320001AE000918F02019F80015FEF48E00E94F8
:10833000AF2D0091B60109930091B7010993009107
:10834000B80109930091B901099314C064E00E9437
:108350006B4212F40C947935012F122F29E0073F5C
:10836000120710F00C94793533272AE00E948743D6
:108370000093C40407E00C949335112321F000917D
:108380008C020C94823563E00E946B42222312F42B
:108390000C9479351093C10406E00C9493351123A5
:1083A00071F010E30091CA04002339F011E30230A8
:1083B00021F012E3013009F013E3199319C00E9470
:1083C000A242043012F00C9479351127002359F0A1
:1083D00012E0013041F011E0023029F013E00330E7
:1083E00011F00C9479351093CA040FEF0093270213
:1083F00004E00C949335112339F010E30091B70495
:1084000000FD11E3199318C00E94A24212F002303D
:1084100014F00C9479351091B704002319F410FF6F
:1084200059F002C010FD41F4F8941091340104E0B9
:10843000102710933501789404E00C9493350027AD
:108440001127222733271BC03091B3042091B40495
:108450001091B5040091B6040A50104020403040FD
:108460000EC03091B3042091B4041091B504009172
:10847000B6048AE0080F80E0181F281F381F3093C9
:10848000B3042093B4041093B5040093B60403E03E
:108490000C949335112381F0332722271127009163
:1084A000DB045FEF48E00E94AF2D0091B801099313
:1084B0000091B90109930CC062E00E946B4212F472
:1084C0000C947935173114F00C9479351093DB0442
:1084D00005E00C949335112722273327442755278D
:1084E0000D9109930E9499420AF1100F251F351F23
:1084F000451F6A95C9F0110F221F331F441F4F9368
:108500003F932F931F93110F221F331F441F110FEF
:10851000221F331F441F0F91100F0F91201F0F9127
:10852000301F0F91401FDCCF002708950FEF00236D
:108530000895005320F00A3010F4002308950FEF3F
:10854000002308950D910993005308950E941F344C
:10855000302F31702D911D910C915FEF48E00E94FA
:10856000AF2D00E30993099309930091B201099398
:108570000091B30109930091B40109930091B501F1
:1085800009930091B60109930091B70109930091F5
:10859000B80109930091B90109930EE00895712F74
:1085A0000D9109930E9499420AF42CC00D910993F0
:1085B0000E9499420AF426C00D9109930E949942A3
:1085C0000AF420C068E00E946B420AF41BC00C91C0
:1085D0000B3309F017C04F933F932F931F93F894D9
:1085E000172F0E941F3411970E7F1F912F913F91DB
:1085F0004F91402B4D933D932D931C9378940EE017
:10860000002308950FEF0023089510E00E941F3407
:10861000402F4E701091C80413FD40930E041D911D
:108620002D913C91AF93BF930F931F932F933F9343
:1086300011E00E941F34402F4E7040930D041D9195
:108640002D913C914F914C934F914E934F914E935E
:108650004F914E93BF91AF913C932E931E930E93E7
:108660000895F89410E00E941F3400918B060E9339
:108670000E7000930D041091C80413FF00930E04B4
:10868000119600918C060D9300918D060D9300912B
:108690008E060D9300918F060D9300919006006851
:1086A0000C930FEF009327020093DE030027009343
:1086B0005402009355020E94063478940895A8014C
:1086C0005A014FE35527BA019A0185010E94874359
:1086D000A8011A01260E371E36942794B101910184
:1086E00085010E948743A8011A01260E371E369481
:1086F0002794B101910185010E948743A8011A01C5
:10870000260E371E36942794B10181010895EE2478
:10871000DD2480E1000F111FEE1CDD1CE216D306E4
:1087200018F0E21AD30A03958A95A1F70895029FDB
:10873000C001129F900D039F900D8C0108959091A0
:10874000C90497708827F8E1EEEB5AE0589FD001F2
:108750005527A90FB51FEA0FFB1F359654919517A2
:1087600009F04CC0D0011496F8E1EEEBEA0FFB1FC4
:1087700054915E33B1F5F8E1EEEBE00DF11D75912A
:108780006591559145910E94F433E4F1C1E04C2F7D
:10879000480F6AE0649FD0015527A90FB51FF8E183
:1087A000EEEBEA0FFB1F359654919517B9F4D00103
:1087B0001496F8E1EEEBEA0FFB1F54915C3371F471
:1087C000F8E1EEEBE00DF11D759165915591459144
:1087D0000E94F433CCF0C1F08C0F10C0C395C630AA
:1087E000B1F65D3359F4F8E1EEEBE00DF11D759152
:1087F0006591559145910E94F43331F0839587320C
:108800000CF4A1CF68940895E8940895B3E0A9E723
:1088100015E100E2F8940D931A95E9F700E2009350
:10882000AB027894089520533AE0329F1053010E22
:108830003327E2E9F8E10A95000FE00FF31F0591F5
:108840001491000D131F0C5110402227552748E0AA
:108850000E94AF2D2091B7011091B8010091B9018C
:1088600008950F7002951127B7E0A9E4A00FB11F7A
:10887000F8E0E0E11CE022270D910C3309F42FEF22
:10888000222309F000E201931A95B1F707E1009362
:108890000804089510E00E941F340E7011E30630A2
:1088A00099F012E3043081F013E3003069F014E32F
:1088B0000A3051F015E3083039F016E30C3021F09E
:1088C00017E3023009F019E3089566E0013399F0E7
:1088D00064E0023381F060E0033369F06AE004335E
:1088E00051F068E0053339F06CE0063321F062E0C6
:1088F000073309F06EE0089500EC00931104F8943A
:108900000091420100640F7D10ED0E946A3378945B
:10891000F89400913B010170006D10E70E946A33EA
:1089200000913801086010E40E944E3306ED0E9469
:108930009E330FEF0E949E33789444E68DE07727B4
:1089400066275527109144011078062F00950F7760
:10895000012B0E948C4510EF0E946A33052F0F7780
:10896000072B0E948C4510EE0E946A330E947645C8
:108970000AF485C04F935F938F930E949E450E9497
:10898000BC450E9420468F915F914F91009102015A
:10899000041738F45093A00660939F067093A106C5
:1089A000402F08170CF472C08894552309F40894DA
:1089B000551F57FFC7CF8894662309F40894661F94
:1089C00067FFBFCF772311F470E8BACF03E0800FC1
:1089D00089310CF4B4CF8DE060919F06669590913B
:1089E0009F06992311F497E003C0990F97FD9FE725
:1089F0005091A00656953091A006332311F437E02C
:108A000003C0330F97FD9FE7109144011078062FA4
:108A100000950F77012B0E948C4510EF0E946A335E
:108A20007091A106052F0F77072B0E948C4510EE41
:108A30000E946A330E94764512F13F934F935F93F1
:108A40008F939F930E949E450E94BC450E942046A2
:108A50009F918F915F914F913F9100910201041777
:108A600028F45093A00660939F06402F081774F0D7
:108A70005395531749F66395691709F0B9CF0FE776
:108A800000939D06002700939E0612C000919F064A
:108A90000E948C4500950F7700939D060091A006DB
:108AA0000E948C450F771091A106012B00939E0622
:108AB000F89400913801086010E40E944E3306EDEE
:108AC0000E949E3300270E949E3300913B0110E7D5
:108AD0000E946A330091420110ED0E946A330091B6
:108AE00011040F7B00931104789408950BE0009318
:108AF00010040091320105FD02C0289408950091F0
:108B000010040023B1F7A894089500931004009175
:108B100010040023E1F70895102F107800FD106471
:108B200001FD106202FD106103FD186004FD146078
:108B300005FD126006FD1160012F0895F894109153
:108B40009A0400919B0478940E94064630936B032C
:108B50000093060110930501309123012091240117
:108B60000217130740F0020F131F16950795109375
:108B70002301009324010895F89410919C0400911E
:108B80009D0478940E94064630936A031093030173
:108B900000930401F8943091A4023323A9F1332700
:108BA0003093A40232E03093A302789430912101F3
:108BB0002091220102171307EAF44091A00250917C
:108BC000A102451709F14093A10289013695279525
:108BD0003695279536952795369527953695279579
:108BE000422F432B09F421E0021B130B4AF4002708
:108BF000112706C0F8943BE43093A0023093A10201
:108C000010932101009322017894089516950795F9
:108C100016950795009F112D2EE2129E110E1F92A0
:108C200029E8129F80012091C8042670243031F079
:108C3000263021F02AE033270E9487433F91089590
:108C40007894112700916A0310932601009327015D
:108C5000000F111F000F111F000F111F000F111F18
:108C6000000F111F000F111F0E945F431F930F93EE
:108C7000112700916B031093280100932901000F25
:108C8000111F000F111F000F111F000F111F000FE8
:108C9000111F000F111F0E945F4330912601209188
:108CA00027010E949743000F111F2F913F910E94AF
:108CB00087433091260120912701020F131F309125
:108CC000280120912901A901020F131F2AE033274F
:108CD0000E9497433091260120912701241B350BD8
:108CE0001AF00901102811F4332721E00E9487436C
:108CF0000F931F931AE0019FF894009202011092C3
:108D0000010178941F910F910A50104010F4002730
:108D10001127102F002728E233270E948743109144
:108D2000340116FF0027009369030895B1E0A0E025
:108D3000F8E0E8E6F8940C9111270E94BD46B1F4E2
:108D40001FEF0E94BD4691F41AEA0E94BD4671F4DD
:108D500015E50E94BD4651F40C931196AE17BF075E
:108D600049F778940AE100935C0208950C93789493
:108D70000AE1019500935C0208951C932C9112174F
:108D800008953091F7063323E1F7D6E0C9EF30E2DA
:108D900039933327222711275FEF48E00E94AF2D38
:108DA0000091B70109930091B80109930091B901AD
:0A8DB000099305E00E949335089531
:00000001FF
